:020000040800F2
:10400000000001209D920008BD850008BF850008C2
:10401000C1850008C3850008C585000800000000B0
:10402000000000000000000000000000C78500083C
:10403000C985000800000000CB850008CD85000878
:10404000E5920008E5920008E5920008E592000874
:10405000E5920008E5920008E5920008E592000864
:10406000E5920008E5920008E5920008D185000875
:10407000E5920008E5920008DD850008E985000862
:10408000E5920008E5920008E5920008E592000834
:10409000E5920008E5920008E5920008E592000824
:1040A000E5920008E5920008E5920008E592000814
:1040B000E5920008E5920008E5920008E592000804
:1040C000E5920008E5920008E5920008E5920008F4
:1040D000E5920008F5850008E5920008E5920008E1
:1040E000E5920008E5920008E5920008E5920008D4
:1040F000E5920008E5920008E5920008E5920008C4
:10410000E5920008E5920008E5920008E5920008B3
:10411000E5920008E592000801860008E592000893
:10412000E5920008E5920008E5920008E592000893
:10413000000000000000000000000000000000007F
:10414000000000000000000000000000000000006F
:10415000000000000000000000000000000000005F
:10416000000000000000000000000000000000004F
:10417000000000000000000000000000000000003F
:10418000000000000000000000000000000000002F
:10419000000000000000000000000000000000001F
:1041A000000000000000000000000000000000000F
:1041B00000000000000000000000000000000000FF
:1041C00000000000000000000000000000000000EF
:1041D00000000000000000000000000000000000DF
:0441E0005FF8E0F1B3
:1041E80010B5054C237833B9044B13B10448AFF329
:1041F80000800123237010BD20040020000000006F
:104208001CBC000808B5034B1BB103490348AFF3B6
:10421800008008BD00000000240400201CBC000829
:10422800034613F8012B002AFBD1181A01387047EE
:10423800D0400B1CD1409C46203AD34018435242F0
:10424800634693401843704781F0004102E000BF85
:1042580083F0004330B54FEA41044FEA430594EA3E
:10426800050F08BF90EA020F1FBF54EA000C55EA79
:10427800020C7FEA645C7FEA655C00F0E2804FEA4A
:104288005454D4EB5555B8BF6D420CDD2C4480EA2C
:10429800020281EA030382EA000083EA010180EA5C
:1042A800020281EA0303362D88BF30BD11F0004FAA
:1042B8004FEA01314FF4801C4CEA113102D04042E0
:1042C80061EB410113F0004F4FEA03334CEA13331B
:1042D80002D0524263EB430394EA050F00F0A78033
:1042E800A4F10104D5F1200E0DDB02FA0EFC22FA2E
:1042F80005F2801841F1000103FA0EF2801843FA22
:1043080005F359410EE0A5F120050EF1200E012A12
:1043180003FA0EFC28BF4CF0020C43FA05F3C01850
:1043280051EBE37101F0004507D54FF0000EDCF1C9
:10433800000C7EEB00006EEB0101B1F5801F1BD372
:10434800B1F5001F0CD349085FEA30004FEA3C0C76
:1043580004F101044FEA445212F5800F80F09A806C
:10436800BCF1004F08BF5FEA500C50F1000041EB70
:10437800045141EA050130BD5FEA4C0C404141EB74
:10438800010111F4801FA4F10104E9D191F0000F9B
:1043980004BF01460020B1FA81F308BF2033A3F11E
:1043A8000B03B3F120020CDA0C3208DD02F1140C15
:1043B800C2F10C0201FA0CF021FA02F10CE002F150
:1043C8001402D8BFC2F1200C01FA02F120FA0CFC49
:1043D800DCBF41EA0C019040E41AA2BF01EB045192
:1043E800294330BD6FEA04041F3C1CDA0C340EDC90
:1043F80004F11404C4F1200220FA04F001FA02F3D3
:1044080040EA030021FA04F345EA030130BDC4F190
:104418000C04C4F1200220FA02F001FA04F340EA85
:104428000300294630BD21FA04F0294630BD94F036
:10443800000F83F4801306BF81F480110134013D1D
:104448004EE77FEA645C18BF7FEA655C29D094EA8E
:10445800050F08BF90EA020F05D054EA000C04BF0C
:104468001946104630BD91EA030F1EBF00210020F7
:1044780030BD5FEA545C05D14000494128BF41F096
:10448800004130BD14F580043CBF01F5801130BDFA
:1044980001F0004545F0FE4141F470014FF0000085
:1044A80030BD7FEA645C1ABF194610467FEA655C36
:1044B8001CBF0B46024650EA013406BF52EA0335D8
:1044C80091EA030F41F4002130BD00BF90F0000FC6
:1044D80004BF0021704730B54FF4806404F1320402
:1044E8004FF000054FF0000150E700BF90F0000FBB
:1044F80004BF0021704730B54FF4806404F13204E2
:1045080010F0004548BF40424FF000013EE700BFB1
:1045180042004FEAE2014FEA31014FEA02701FBF41
:1045280012F07F4393F07F4F81F06051704792F013
:10453800000F14BF93F07F4F704730B54FF460748D
:1045480001F0004521F0004120E700BF50EA0102D8
:1045580008BF704730B54FF000050AE050EA010285
:1045680008BF704730B511F0004502D5404261EBF5
:1045780041014FF4806404F132045FEA915C3FF436
:10458800DCAE4FF003025FEADC0C18BF03325FEACF
:10459800DC0C18BF033202EBDC02C2F1200300FA84
:1045A80003FC20FA02F001FA03FE40EA0E0021FAA9
:1045B80002F11444C1E600BF70B54FF0FF0C4CF493
:1045C800E06C1CEA11541DBF1CEA135594EA0C0F49
:1045D80095EA0C0F00F0DEF82C4481EA030621EA84
:1045E8004C5123EA4C5350EA013518BF52EA0335BF
:1045F80041F4801143F4801338D0A0FB02CE4FF071
:104608000005E1FB02E506F00042E0FB03E54FF0A0
:104618000006E1FB03569CF0000F18BF4EF0010E98
:10462800A4F1FF04B6F5007F64F5407404D25FEA94
:104638004E0E6D4146EB060642EAC62141EA555147
:104648004FEAC52040EA5E504FEACE2EB4F1FD0C89
:1046580088BFBCF5E06F1ED8BEF1004F08BF5FEA07
:10466800500E50F1000041EB045170BD06F00046B9
:1046780046EA010140EA020081EA0301B4EB5C0466
:10468800C2BFD4EB0C0541EA045170BD41F480115E
:104698004FF0000E013C00F3AB8014F1360FDEBF83
:1046A800002001F0004170BDC4F10004203C35DA5F
:1046B8000C341BDC04F11404C4F1200500FA05F3E2
:1046C80020FA04F001FA05F240EA020001F0004283
:1046D80021F0004110EBD37021FA04F642EB0601F9
:1046E8005EEA430E08BF20EAD37070BDC4F10C0423
:1046F800C4F1200500FA04F320FA05F001FA04F2E7
:1047080040EA020001F0004110EBD37041F10001D2
:104718005EEA430E08BF20EAD37070BDC4F12005DD
:1047280000FA05F24EEA020E20FA04F301FA05F245
:1047380043EA020321FA04F001F0004121FA04F2ED
:1047480020EA020000EBD3705EEA430E08BF20EABD
:10475800D37070BD94F0000F0FD101F000464000F7
:1047680041EB010111F4801F08BF013CF7D041EA79
:10477800060195F0000F18BF704703F0004652007D
:1047880043EB030313F4801F08BF013DF7D043EA4E
:104798000603704794EA0C0F0CEA135518BF95EA04
:1047A8000C0F0CD050EA410618BF52EA4306D1D18B
:1047B80081EA030101F000414FF0000070BD50EAAA
:1047C800410606BF1046194652EA430619D094EA34
:1047D8000C0F02D150EA013613D195EA0C0F05D11E
:1047E80052EA03361CBF104619460AD181EA030172
:1047F80001F0004141F0FE4141F470014FF000002A
:1048080070BD41F0FE4141F4780170BD70B54FF0C4
:10481800FF0C4CF4E06C1CEA11541DBF1CEA135544
:1048280094EA0C0F95EA0C0F00F0A7F8A4EB050426
:1048380081EA030E52EA03354FEA013100F088801D
:104848004FEA03334FF0805545EA131343EA1263E6
:104858004FEA022245EA111545EA10654FEA00269B
:104868000EF000419D4208BF964244F1FD0404F554
:10487800407402D25B084FEA3202B61A65EB0305B0
:104888005B084FEA32024FF480104FF4002CB6EB6D
:10489800020E75EB030E22BFB61A754640EA0C00ED
:1048A8005B084FEA3202B6EB020E75EB030E22BF2D
:1048B800B61A754640EA5C005B084FEA3202B6EB6E
:1048C800020E75EB030E22BFB61A754640EA9C002D
:1048D8005B084FEA3202B6EB020E75EB030E22BFFD
:1048E800B61A754640EADC0055EA060E18D04FEABB
:1048F800051545EA16754FEA06164FEAC30343EA5B
:1049080052734FEAC2025FEA1C1CC0D111F4801F27
:104918000BD141EA00014FF000004FF0004CB6E720
:1049280011F4801F04BF01430020B4F1FD0C88BFBF
:10493800BCF5E06F3FF6AFAEB5EB030C04BFB6EBCA
:10494800020C5FEA500C50F1000041EB045170BDBD
:104958000EF0004E4EEA113114EB5C04C2BFD4EBEA
:104968000C0541EA045170BD41F480114FF0000E6E
:10497800013C90E645EA060E8DE60CEA135594EAEA
:104988000C0F08BF95EA0C0F3FF43BAF94EA0C0FED
:104998000AD150EA01347FF434AF95EA0C0F7FF462
:1049A80025AF104619462CE795EA0C0F06D152EAB6
:1049B80003353FF4FDAE1046194622E750EA41069A
:1049C80018BF52EA43067FF4C5AE50EA41047FF4AB
:1049D8000DAF52EA43057FF4EBAE12E74FF0FF3C10
:1049E80006E000BF4FF0010C02E000BF4FF0010CE1
:1049F8004DF804CD4FEA410C7FEA6C5C4FEA430C5A
:104A080018BF7FEA6C5C1BD001B050EA410C0CBFA8
:104A180052EA430C91EA030F02BF90EA020F00200A
:104A2800704710F1000F91EA030F58BF994208BF71
:104A380090422CBFD8176FEAE37040F0010070472E
:104A48004FEA410C7FEA6C5C02D150EA013C07D185
:104A58004FEA430C7FEA6C5CD6D152EA033CD3D0D0
:104A68005DF8040B704700BF8446104662468C46CA
:104A78001946634600E000BF01B5FFF7B7FF0028FD
:104A880048BF10F1000F01BD4DF808EDFFF7F4FF26
:104A98000CBF012000205DF808FB00BF4DF808EDB1
:104AA800FFF7EAFF34BF012000205DF808FB00BFD4
:104AB8004DF808EDFFF7E0FF94BF012000205DF8F6
:104AC80008FB00BF4DF808EDFFF7CEFF94BF0120AB
:104AD80000205DF808FB00BF4DF808EDFFF7C4FFA4
:104AE80034BF012000205DF808FB00BF4FEA410CED
:104AF8007FEA6C5C02D150EA013C0AD14FEA430CD0
:104B08007FEA6C5C02D152EA033C02D14FF000000C
:104B180070474FF0010070474FEA410212F500124A
:104B280015D211D56FF47873B3EB625212D94FEAEC
:104B3800C12343F0004343EA505311F0004F23FAD6
:104B480002F018BF404270474FF00000704750EA2B
:104B5800013005D111F0004008BF6FF000407047E8
:104B68004FF00000704700BF4A0011D212F5001242
:104B780011D20DD56FF47873B3EB62520ED44FEAAD
:104B8800C12343F0004343EA505323FA02F070472D
:104B98004FF00000704750EA013002D14FF0FF306B
:104BA80070474FF0000070474FEA4102B2F1E0430E
:104BB80024BFB3F5001CDCF1FE5C0DD901F0004CFC
:104BC8004FEAC0024CEA5070B2F1004F40EB83004C
:104BD80008BF20F00100704711F0804F21D113F178
:104BE8003872BCBF01F00040704741F480114FEAB1
:104BF8005252C2F11802C2F1200C10FA0CF320FA3A
:104C080002F018BF40F001004FEAC1234FEAD32356
:104C180003FA0CFC40EA0C0023FA02F34FEA4303C0
:104C2800CCE77FEA625307D150EA01331EBF4FF049
:104C3800FE4040F44000704701F0004040F0FE4064
:104C480040F40000704700BF80F0004002E000BF61
:104C580081F0004142001FBF5FEA410392EA030F5F
:104C68007FEA226C7FEA236C6AD04FEA1262D2EBA9
:104C78001363C1BFD218414048404140B8BF5B42AE
:104C8800192B88BF704710F0004F40F4000020F047
:104C98007F4018BF404211F0004F41F4000121F05D
:104CA8007F4118BF494292EA030F3FD0A2F10102A7
:104CB80041FA03FC10EB0C00C3F1200301FA03F1E5
:104CC80000F0004302D5494260EB4000B0F5000F08
:104CD80013D3B0F1807F06D340084FEA310102F1C7
:104CE8000102FE2A51D2B1F1004F40EBC25008BF79
:104CF80020F0010040EA03007047490040EB000043
:104D080010F4000FA2F10102EDD1B0FA80FCACF171
:104D1800080CB2EB0C0200FA0CF0AABF00EBC25070
:104D280052421843BCBFD0401843704792F0000F5E
:104D380081F4000106BF80F400000132013BB5E7B1
:104D48004FEA41037FEA226C18BF7FEA236C21D027
:104D580092EA030F04D092F0000F08BF084670478C
:104D680090EA010F1CBF0020704712F07F4F04D15A
:104D7800400028BF40F00040704712F100723CBF6D
:104D880000F50000704700F0004343F0FE4040F497
:104D9800000070477FEA226216BF08467FEA236355
:104DA8000146420206BF5FEA412390EA010F40F440
:104DB800800070474FF0000304E000BF10F000438C
:104DC80048BF40425FEA000C08BF704743F0964373
:104DD80001464FF000001CE050EA010208BF70478E
:104DE8004FF000030AE000BF50EA010208BF704715
:104DF80011F0004302D5404261EB41015FEA010C2A
:104E080002BF84460146002043F0B64308BFA3F121
:104E18008053A3F50003BCFA8CF2083AA3EBC25303
:104E280010DB01FA02FC634400FA02FCC2F1200222
:104E3800BCF1004F20FA02F243EB020008BF20F059
:104E48000100704702F1200201FA02FCC2F12002BF
:104E580050EA4C0021FA02F243EB020008BF20EAB4
:104E6800DC7070474FF0FF0C1CEAD0521EBF1CEAE2
:104E7800D15392EA0C0F93EA0C0F6FD01A4480EAD0
:104E8800010C400218BF5FEA41211ED04FF00063B9
:104E980043EA501043EA5111A0FB01310CF00040E5
:104EA800B1F5000F3EBF490041EAD3715B0040EA0B
:104EB800010062F17F02FD2A1DD8B3F1004F40EBDB
:104EC800C25008BF20F00100704790F0000F0CF0AE
:104ED800004C08BF49024CEA502040EA51207F3A72
:104EE800C2BFD2F1FF0340EAC250704740F400004D
:104EF8004FF00003013A5DDC12F1190FDCBF00F03E
:104F080000407047C2F10002410021FA02F1C2F1EB
:104F1800200200FA02FC5FEA310040F1000053EA87
:104F28004C0308BF20EADC70704792F0000F00F0D5
:104F3800004C02BF400010F4000F013AF9D040EADB
:104F48000C0093F0000F01F0004C02BF490011F46F
:104F5800000F013BF9D041EA0C018FE70CEAD1536D
:104F680092EA0C0F18BF93EA0C0F0AD030F0004CED
:104F780018BF31F0004CD8D180EA010000F00040A1
:104F8800704790F0000F17BF90F0004F084691F05F
:104F9800000F91F0004F14D092EA0C0F01D1420299
:104FA8000FD193EA0C0F03D14B0218BF084608D162
:104FB80080EA010000F0004040F0FE4040F40000AC
:104FC800704740F0FE4040F4400070474FF0FF0C3F
:104FD8001CEAD0521EBF1CEAD15392EA0C0F93EA86
:104FE8000C0F69D0A2EB030280EA010C49024FEAD8
:104FF800402037D04FF0805343EA111143EA101391
:105008000CF000408B4238BF5B0042F17D024FF448
:10501800000C8B4224BF5B1A40EA0C00B3EB510F23
:1050280024BFA3EB510340EA5C00B3EB910F24BF0C
:10503800A3EB910340EA9C00B3EBD10F24BFA3EB91
:10504800D10340EADC001B0118BF5FEA1C1CE0D159
:10505800FD2A3FF650AF8B4240EBC25008BF20F00C
:10506800010070470CF0004C4CEA50207F32C2BF60
:10507800D2F1FF0340EAC250704740F400004FF0FD
:105088000003013A37E792F0000F00F0004C02BF2E
:10509800400010F4000F013AF9D040EA0C0093F0F8
:1050A800000F01F0004C02BF490011F4000F013B52
:1050B800F9D041EA0C0195E70CEAD15392EA0C0FBA
:1050C80008D142027FF47DAF93EA0C0F7FF470AFF2
:1050D800084676E793EA0C0F04D14B023FF44CAF35
:1050E80008466EE730F0004C18BF31F0004CCAD1CA
:1050F80030F000427FF45CAF31F000437FF43CAF06
:105108005FE700BF42000ED2B2F1FE4F0BD34FF063
:105118009E03B3EB126209D44FEA002343F0004325
:1051280023FA02F070474FF00000704712F1610F48
:1051380001D1420202D14FF0FF3070474FF000001A
:10514800704700BF38B50E4B054618784FF47A7390
:10515800B3FBF0F30B4A1068B0FBF3F000F038FB38
:10516800044658B90F2D09D8024629464FF0FF309A
:1051780000F0EEFA044B20461D6038BD012038BD12
:10518800000000201802002004000020074A08B58B
:105198001368032043F01003136000F0C7FA0020DF
:1051A800FFF7D0FF03F0F4F8002008BD002002400C
:1051B800034A044B11681B780B441360704700BF07
:1051C8007804002000000020014B1868704700BFD9
:1051D8007804002038B50446FFF7F6FF0546631C3F
:1051E8001EBF044B1B78E418FFF7EEFF401B8442F8
:1051F800FAD838BD000000207047436A10B59A6A93
:1052080012F0500F1BD19A6A42F400729A621A681F
:10521800926802F46022B2F5602F0CD1DA6852B9B4
:105228009A6A22F480729A629A6AD2045EBF9A6A73
:1052380042F001029A621846FFF7DEFF10BD1B6AB2
:10524800BDE810401B6B1847704708B5406AFFF768
:10525800FBFF08BD7047406A08B5836A43F0400306
:105268008362C36A43F00403C362FFF7F3FF08BD18
:10527800002373B5019390F82430012B74D00123D7
:105288004D6880F82430062D02684FEA85030C68C3
:1052980025D82B441F25566B053B9D4026EA05055E
:1052A80004FA03F32B435363092C4FEA44038D6834
:1052B8002FD907262344D1681E3B9E4021EA0601C8
:1052C80005FA03F30B43D360A4F11003012B2BD988
:1052D8000023002280F82420184602B070BD0C2D4F
:1052E8000BD82B441F25166B233B9D4026EA05054A
:1052F80004FA03F32B431363D6E72B441F25D66A1E
:10530800413B9D4026EA050504FA03F32B43D3628B
:10531800CAE70726116923449E4021EA060105FAD7
:1053280003F30B431361CFE7104B9A4216D19368EE
:105338001B02CDD49368102C43F400039360C7D1AB
:105348000B4B0C4A1B68B3FBF2F20A23534301933D
:10535800019B002BBCD0019B013BF8E7836A43F01B
:10536800200383620123B4E70223B5E70024014048
:105378001802002040420F00002373B50193036810
:1053880004469A68D20702D5002002B070BD9A6818
:1053980042F001029A60124B124A1B68B3FBF2F307
:1053A8000193019BC3B9FFF70FFF064623689D6869
:1053B80015F00105E8D1FFF707FF801B0228F5D992
:1053C800A36A84F8245043F01003A362E36A01201F
:1053D80043F00103E362D8E7019B013BE0E700BF2C
:1053E8001802002040420F002DE9D8419046404B5A
:1053F800026804469A420F4602D03E498A4203D1C7
:105408005B6813F4702F6ED194F82430012B6CD0A4
:105418000123204684F82430FFF7AEFF0646002813
:105428005DD1A06A216820F47060324B20F0010041
:1054380040F480709942A06204D12D4A536813F455
:10544800702F3ED1A36A23F48013A3624B685A05D8
:1054580005D5A36A23F4405343F48053A362A36A97
:10546800206A13F4805318BFE36A3A4618BF23F042
:105478000603E362002384F824301F4B4C31836217
:105488001E4BC3621E4B03636FF0020341F84C3C92
:1054980051F8443C43F4807341F8443C434600F0DF
:1054A800EDF923689A6802F46022B2F5602F9A68D1
:1054B8000CBF42F4A00242F480129A603046BDE864
:1054C800D881A36A43F48013A36253685B0541BF84
:1054D800A06A20F4405040F48050A062BFE7002347
:1054E80084F82430EAE70126E8E70226E6E700BF69
:1054F80000240140002801400352000853520008CC
:105508005F52000838B5036804469A68D20701D488
:10551800002038BD9A6822F001029A60FFF754FE15
:10552800054623689B68DB07F2D5FFF74DFE401B55
:105538000228F6D9A36A012043F01003A362E36AA4
:1055480043F00103E36238BDF8B50446002877D07C
:10555800836A23B9C36280F8243002F03BFF2046F7
:10556800FFF7D0FFA36A13F010036BD1002869D1AD
:10557800A26A374922F4885222F0020242F002025B
:10558800A26294E824008A42E16904D1B1F5402F6F
:1055980008BF4FF40021E66845EA46052943A56897
:1055A800B5F5807F35D0012D08BF4FF4807367694A
:1055B800012F06D17EBBA669013E43EA463343F478
:1055C80000635668B5F5807F26F4694643EA06030A
:1055D800536096681F4B03EA060343EA010393608E
:1055E80001D0012D20D12369013B1B05D56A25F483
:1055F80070052B43D3629268174B1340994215D11B
:105608000023E362A36A23F0030343F00103A362C8
:10561800F8BD2B46CBE7A66A46F02006A662E66AE6
:1056280046F00106E662CCE70023DFE7A36A23F031
:10563800120343F01003A362E36A43F00103E36239
:105648000120F8BDA36A43F01003A362F8E700BF86
:10565800003C0140FDF7E1FFFE0E1FFF002373B57C
:10566800019390F824300446012B5AD0012380F886
:105678002430FFF747FF0546002832D1A36A0220ED
:1056880023F4885323F0020343F00203A362264B5A
:105698001E6800F0AFFFB6FBF0F040000190019BE0
:1056A8001BBB2046FFF768FE2268936843F0080397
:1056B8009360FFF789FD064623689A68120718D495
:1056C8009A6842F004029A60FFF77EFD0646236856
:1056D8009B685B071FD4A36A23F0030343F001030D
:1056E800A362002384F8243012E0019B013B01935C
:1056F800D5E7FFF769FD801B0A28DDD9A36A0125D4
:1057080023F0120343F01003A362002384F824302B
:10571800284602B070BDFFF757FD801B0A28D6D96E
:10572800ECE70225F4E700BF18020020074A000250
:10573800D36800F4E06023F4E0631B041B0C43F01F
:10574800BF6343F400330343D360704700ED00E0C8
:10575800174B30B5DC68C4F30224C4F10703251DD8
:10576800042B28BF0423062D4FF0010598BF002401
:1057780005FA03F303F1FF3388BF033C1940A14046
:1057880005FA04F4013C2240002842EA01024FEAEB
:105798000212AFBF00F16040064B00F00F00D2B21A
:1057A800A5BFD2B200F561401A5480F8002330BD7D
:1057B80000ED00E014ED00E00123420900F01F00B5
:1057C80003FA00F0014B43F82200704700E100E0C3
:1057D8000138B0F1807F0AD2F021064B064A5860A2
:1057E80082F823100020072298601A607047012071
:1057F800704700BF10E000E000ED00E010B50028A1
:1058080032D00168194B1424994225D8184AA3F2BA
:1058180007430A44B2FBF4F2920002648468C3634B
:1058280043680A682343C46822F47F522343046907
:1058380022F0300223434469234384692343C46923
:10584800234313430B600122002380F82120836344
:1058580080F82030184610BD064B0B44B3FBF4F318
:105868009B000364044BD9E7012010BD07040240E4
:10587800F8FFFDBFF8FBFDBF00040240F0B590F84B
:105888002040012C35D0012490F8215080F8204088
:10589800A5424FF000064FF0020428D180F82140BD
:1058A800046886632668076C26F001062660C66BC6
:1058B800BD407560636043680568102BC36A0BBF01
:1058C800A260A160E160E2604BB1236843F00E037F
:1058D80023602B68002043F001032B60F0BD236890
:1058E80023F004032360236843F00A03F0E780F8F9
:1058F80020600220F0BD000090F8213010B5022B86
:1059080003D004238363012010BD03681A6822F0C2
:105918000E021A601A6822F001021A60294A93429C
:1059280024D902F56272934219D01432934218D0E6
:105938001432934217D0143293420CBF4FF4805361
:105948004FF48033204A53600123002480F821302B
:10595800436B80F820409BB39847204610BD012335
:10596800F0E71023EEE74FF48073EBE717498B421B
:1059780016D014318B4215D014318B4214D0143107
:105988008B4214D014318B4214D014318B4214D072
:10599800934214BF4FF480334FF080730C4AD2E720
:1059A8000123FBE71023F9E74FF48073F6E74FF480
:1059B8008053F3E74FF48033F0E74FF48013EDE7BB
:1059C800184610BD80000240000402400800024052
:1059D8000000024070B40425C66B026C346803688A
:1059E80095402542196855D04D0753D51A68960633
:1059F8005EBF1A6822F004021A60604A93421FD9F7
:105A080002F56272934214D01432934213D01432C6
:105A1800934212D0143293420CBF4FF480434FF498
:105A28008023574A5360C36A002B00F0A58070BCDE
:105A380018470423F5E74023F3E74FF48063F0E7C2
:105A480050498B4216D014318B4215D014318B42F9
:105A580014D014318B4214D014318B4214D0143129
:105A68008B4214D0934214BF4FF480234FF08063CD
:105A7800454AD7E70423FBE74023F9E74FF480635F
:105A8800F6E74FF48043F3E74FF48023F0E74FF451
:105A98008003EDE702259540254257D08D0755D55F
:105AA8001A68940606D41A6822F00A021A600122BB
:105AB80080F82120314A93421ED902F5627293423E
:105AC80013D01432934212D01432934211D01432AC
:105AD80093420CBF4FF400534FF40033284A5360ED
:105AE800002380F82030836A9EE70223F6E720230C
:105AF800F4E74FF40073F1E722498B4216D01431D2
:105B08008B4215D014318B4214D014318B4214D0EF
:105B180014318B4214D014318B4214D0934214BFE9
:105B28004FF400334FF00073174AD8E70223FBE71E
:105B38002023F9E74FF40073F6E74FF40053F3E737
:105B48004FF40033F0E74FF40013EDE708259540D4
:105B5800254211D009070FD5196821F00E011960E7
:105B6800012303FA02F27260836380F82130002374
:105B780080F82030036B57E770BC70478000024004
:105B8800000402400800024000000240114AD368A5
:105B980013F0100305D01049CB6943F00203CB6121
:105BA8001023D268500706D50B4943F00403CA698D
:105BB80042F00102CA61074AD169C90708D50648F7
:105BC800C16941F00401C161D16921F00101D161CC
:105BD800D36070470020024080040020064B1869FB
:105BE80010F0800007D0054A5A6002F188325A60E6
:105BF8001869C0F3C01070470020024023016745B0
:105C0800034A0020136943F080031361704700BF03
:105C180000200240F8B50646FFF7D6FA114C0746B1
:105C28002546E368D80712D4E368990644BF2023C1
:105C3800E360EB68DA0606D4EB69DB0703D4E868AF
:105C480010F0040002D0FFF7A1FF0120F8BD731C7B
:105C5800E7D00EB90320F8BDFFF7B6FAC01B86429D
:105C6800DFD2F7E7002002402DE9F84F1F4C994694
:105C7800237E0546012B0F46904633D001234CF274
:105C880050302376FFF7C6FF40BB012D03D0022D0D
:105C98000CBF022504250026B246DFF854B03201B5
:105CA80040464946FEF7C4FAC4F81CA0DBF8103099
:105CB80080B243F00103CBF8103027F816004CF2FD
:105CC8005030FFF7A7FFDBF8103023F00103CBF8C3
:105CD800103018B90136F3B29D42E0D8002323767C
:105CE800BDE8F88F0220BDE8F88F00BF80040020CF
:105CF800002002400022064BDA61064B1A6942F086
:105D080004021A611A6942F040021A61704700BF22
:105D180080040020002002400022064BDA61064B76
:105D28001A6942F002021A6158611A6942F0400287
:105D38001A61704780040020002002402DE9F041DC
:105D4800234D07462B7E8846012B3DD0012403684E
:105D58002C76022B4CF2503013D1FFF75BFF20B1A9
:105D6800012000232B76BDE8F081FFF7C3FF4CF23A
:105D78005030FFF74FFF174A136923F004031361EC
:105D8800EFE7FFF747FF0028EAD14FF0FF33C8F8E5
:105D980000302046BE680F4CFA68BB6803EBC2238C
:105DA8009E42DED23046FFF7B7FF4CF25030FFF785
:105DB80031FF236923F00203236110B1C8F80060A2
:105DC800CFE706F50066E7E70220BDE8F08100BFEF
:105DD80080040020002002402DE9F74F00221646DB
:105DE8006C4F6D4BDFF8B8E1DFF8B8C14FF0010830
:105DF8000C6808FA06F808EA0404A04540F0858013
:105E08004D68122D00F0B78000F28D80022D00F051
:105E1800AF8000F28180002D00F09180012D00F00C
:105E2800A5804FF00F09FF2C93BF824606F18045ED
:105E3800083DD0F800B092BFB500D0F804B0AD006E
:105E480009FA05F82BEA080802FA05F588BF00F1F7
:105E5800040A48EA0505CAF80050D1F804A01AF067
:105E6800805F52D0BD6926F0030845F00105BD6189
:105E7800BD6908F1804805F00105019508F58038ED
:105E880006F0030B019D4FEA8B0BD8F8085009FA6E
:105E98000BF925EA0909414DA84271D005F580653D
:105EA800A8426FD005F58065A8426DD005F58065DC
:105EB800A8426BD005F58065A84269D070450CBF33
:105EC8000525062505FA0BF545EA0905C8F8085021
:105ED8001D681AF4803F14BF2543A5431D605D6803
:105EE8001AF4003F14BF2543A5435D609D681AF46A
:105EF800801F14BF2543A5439D60DD681AF4001F69
:105F080014BF2C4325EA0404DC600136102E7FF40C
:105F18006DAF03B0BDE8F08F032D25D0112D80D1D2
:105F2800CA6804327DE7654509D012D8DFF8789051
:105F38004D4504D009F580394D457FF472AF8A6824
:105F4800E2B1012A0CBFC0F81080C0F81480082202
:105F580067E7DFF858904D45F1D009F580394D4590
:105F6800EDD0A9F58019E7E700225AE7CA6858E793
:105F7800CA68083255E7CA680C3252E7042250E76B
:105F880000259FE701259DE702259BE7032599E763
:105F9800042597E700100240000401400008014072
:105FA800001C0140000021100000111000003110F9
:105FB8008368194214BF0120002070470AB10161AB
:105FC80070470904FBE7C3685940C1607047000087
:105FD80003682DE9F341DB07054610D42B689F07BA
:105FE8005ED42B68190700F195802B685A0700F1D9
:105FF800BF80EA69002A40F02D81002014E0904C0F
:10600800636803F00C03042B07D0636803F00C03E8
:10601800082B0CD16368DE0309D523689C03DDD502
:106028006B68002BDAD1012002B0BDE8F0816B6803
:10603800B3F5803F10D1236843F480332360FFF722
:10604800C3F8064623689803C8D4FFF7BDF8801B39
:106058006428F7D90320E7E79BB9236823F4803342
:106068002360236823F480232360FFF7ADF80646F6
:1060780023689903B2D5FFF7A7F8801B6428F7D9DE
:10608800E8E7B3F5A02F236803D143F48023236006
:10609800D1E723F480332360236823F48023CDE7FA
:1060A800674C636813F00C0F07D0636803F00C03A8
:1060B800082B10D16368DA030DD423689B0702D537
:1060C8002B69012BAFD123686A6923F0F80343EAEF
:1060D800C203236085E72A695A4B6AB101221A6014
:1060E800FFF772F8064623689F07ECD4FFF76CF8B1
:1060F800801B0228F7D9ADE71A60FFF765F8064656
:10610800236898077FF56DAFFFF75EF8801B0228BC
:10611800F6D99FE7AA694A4C4B4BDAB101221A60BB
:10612800FFF752F80646636A9B070DD54FF4FA52FB
:10613800464B1B68B3FBF2F3019300BF019B5A1E49
:106148000192002BF9D150E7FFF73EF8801B022897
:10615800E9D97FE71A60FFF737F80646636A9F07B1
:106168007FF543AFFFF730F8801B0228F6D971E7B7
:10617800334CE369D80024D40127E36943F0805302
:10618800E361E36903F080530093009B304E33686A
:10619800D90518D5EB68012B26D1236A43F00103F2
:1061A8002362FFF711F841F288368046236A9B077D
:1061B8003FD5002F3FF41DAFE36923F08053E3611F
:1061C80017E70027E2E7336843F480733360FEF78C
:1061D800FBFF80463368DA05DCD4FEF7F5FFA0EB59
:1061E80008006428F6D935E7ABB9236A41F2883844
:1061F80023F001032362236A23F004032362FEF7DA
:10620800E3FF0646236A9807D3D5FEF7DDFF801B18
:106218004045F7D91EE7052B236A03D143F0040351
:106228002362BAE723F001032362236A23F00403FD
:10623800B6E7FEF7C9FFA0EB0800B042B6D909E7F8
:10624800001002400000424280044242180200202E
:1062580000700040224C636803F00C03082B3FF4E5
:10626800E2AE00231F4E022A33602BD1FEF7ACFFAB
:106278000746236899011FD42B6AB3F5803F05D1DF
:106288006268A96822F400320A436260696A626837
:106298000B4322F474121343636001233360FEF747
:1062A80093FF054623689A013FF5A7AEFEF78CFFDA
:1062B800401B0228F6D9CDE6FEF786FFC01B022850
:1062C800D7D9C7E6FEF780FF054623689B017FF50F
:1062D80094AEFEF779FF401B0228F6D9BAE600BF54
:1062E800001002406000424230B5194B87B002AC42
:1062F80003F11005224618685968083303C2AB42F7
:106308001446F7D101238DF80430022311498DF882
:1063180005304B6803F00C02082A17D1C3F38342F7
:1063280006A80244DB0312F8102C0CD54B680A4867
:10633800C3F34043504306AA134413F8143CB0FB7C
:10634800F3F007B030BD05485043FAE70248F8E7D4
:1063580038BC00080010024000127A0000093D0015
:10636800544A2DE9F0411368054603F007038B42B0
:106378000E462AD329688C0734D4CA0747D44D4A15
:10638800136803F007039E42C0F082802A684A4CD3
:1063980012F0040F40F08780130706D563682A6956
:1063A80023F4605343EAC2036360FFF79DFF636809
:1063B800424AC3F30313D35CD840414B1860002012
:1063C800FEF7C0FE0020BDE8F081136823F0070344
:1063D8000B431360136803F007039942CAD00120E6
:1063E800BDE8F081344B11F0040F1EBF5A6842F427
:1063F800E0625A60080742BF5A6842F460525A6025
:106408005A68A86822F0F00202435A60B5E76A6841
:10641800294C012A23681CD113F4003FDFD063689C
:1064280041F2883823F0030313436360FEF7CCFE80
:106438006B680746012B14D1636803F00C03042B27
:106448009DD0FEF7C1FEC01B4045F5D90320BDE82D
:10645800F081022A02D113F0007FDFE713F0020F68
:10646800DCE7022B0FD1636803F00C03082B86D0FE
:10647800FEF7AAFEC01B4045F5D9E7E7FEF7A4FEE4
:10648800C01B4045E2D8636813F00C0FF6D176E7DD
:10649800136823F0070333431360136803F00703FB
:1064A8009E429CD172E76368E96823F4E0630B437A
:1064B800636071E70020024000100240F2BC00084F
:1064C80018020020044B054A5B68C3F30223D35C1F
:1064D800034A1068D84070470010024002BD000807
:1064E80018020020044B054A5B68C3F3C223D35C3F
:1064F800034A1068D84070470010024002BD0008E7
:106508001802002003682DE9F341D907054620D574
:10651800354CE369DA0032D40127E36943F080534C
:10652800E361E36903F080530193019B2F4E3368C5
:10653800DB0526D5236A13F4407336D1236A6A68CB
:1065480023F44073134323621FB1E36923F080539C
:10655800E3612868830706D5234AA968536823F4AA
:1065680040430B43536010F010001BD01E4A69696A
:106578005368002023F480030B43536012E0002784
:10658800D4E7336843F480733360FEF71DFE80461A
:106598003368D805CED4FEF717FEA0EB08006428B0
:1065A800F6D9032002B0BDE8F0816A6802F44072AF
:1065B8009342C3D001200E4A236A1060002023F4BE
:1065C800407110602162D907B8D5FEF7FDFD41F290
:1065D80088380646236A9A07B0D4FEF7F5FD801B73
:1065E8004045F7D9DDE700BF0010024000700040C9
:1065F80040044242024670B53B4B86B002AD03F1FF
:1066080010062C4618685968083303C4B342254657
:10661800F7D101238DF804300223501E8DF8053080
:106628000F285ED8DFE800F032515D2D5D5D5D2DED
:106638005D5D5D5D5D5D5D082C4B5968186810F007
:10664800807037D0C1F3834206A8024412F8100CB8
:10665800CA0341BF5A6806A9C2F34042521844BF50
:1066680012F8141C224A5B684CBFB2FBF1F2214AB3
:106678005B0202FB00F01DD403234000B0FBF3F0E3
:1066880018E006B0BDE87040FFF72EBE40F20231B8
:10669800164A136A1940B1F5817F1FD003F440737D
:1066A800B3F5007F08D149F64040536A13F0020F52
:1066B80008BF002006B070BDB3F5407F11D1136844
:1066C8004FF2244013F4003FF2E7FFF70BFF074BAC
:1066D8005B68C3F3813301335B00CFE74FF40040BD
:1066E800E8E70020E6E700BF48BC000800100240C9
:1066F80000127A0000093D007047704770477047E4
:10670800036810B51A69044691070ED5DA6892072E
:106718000BD56FF002021A6101229B6902779B0771
:1067280077D0FFF7EAFF0023237723681A69500719
:1067380010D5DA6851070DD56FF004021A610222EC
:106748009B69227713F4407F204668D0FFF7D5FF76
:106758000023237723681A6912070FD5DA68100710
:106768000CD56FF008021A610422DB6922779907B9
:1067780020465AD0FFF7C1FF0023237723681A6900
:10678800D20610D5DA68D0060DD56FF010021A615E
:106798000822DB69227713F4407F20464BD0FFF7AD
:1067A800ACFF0023237723681A69D10708D5DA6874
:1067B800D20705D56FF0010220461A6101F058FA98
:1067C80023681A69100608D5DA68110605D56FF02E
:1067D800800220461A6100F0BEF823681A69520642
:1067E80008D5DA68500605D56FF0400220461A61D0
:1067F800FFF785FF23681A69910622D5DA689206A1
:106808001FD56FF020022046BDE810401A6100F045
:10681800A1B8FFF771FF2046FFF770FF83E7FFF786
:106828006BFF2046FFF76AFF92E7FFF765FF2046F8
:10683800FFF764FFA0E7FFF75FFF2046FFF75EFF63
:10684800AFE710BD244A0368904212D002F50062F7
:1068580090420ED0B0F1804F0BD0A2F59832904202
:1068680007D002F58062904203D002F58062904220
:106878001DD14A6823F070031343174A904212D07F
:1068880002F5006290420ED0B0F1804F0BD0A2F515
:106898009832904207D002F58062904203D002F508
:1068A8008062904203D1CA6823F4407313434A6953
:1068B80023F08003134303608B68C3620B68836211
:1068C800054B984203D003F50063984201D10B6948
:1068D8000363012343617047002C014010B504464F
:1068E800A0B190F83D3003F0FF021BB980F83C20BE
:1068F80001F0E0FD0223206884F83D30211DFFF7F8
:10690800A1FF0123002084F83D3010BD012010BDF7
:1069180090F83C3010B5012B4FF0020318D080F8E6
:106928003D3003680C685A68496822F070025A6062
:106938005A6822435A609A6822F080029A609A68DC
:106948000A439A60012380F83D30002380F83C30E8
:10695800184610BD704770470368DA6822F49072D1
:10696800DA605A6922F001025A61202380F83A302D
:10697800704700002DE9F0470568C2682B69016976
:1069880023F4405313432B618368EA680B4341693E
:1069980022F4B05222F00C020B431343EB606B69F4
:1069A800826923F4407313436B61404B81469D42D7
:1069B8004FF0190446D1FFF795FD04FB00F3D9F811
:1069C80004604FF06408B600B3FBF6F3B3FBF8F3CA
:1069D8001E01FFF787FD6043D9F804309B00B0FB28
:1069E800F3F7FFF77FFD6043D9F804309B00B0FB55
:1069F800F3F3B3FBF8F308FB13731B013233B3FB58
:106A0800F8F303F0F007FFF76DFD6043D9F80420B1
:106A18009200B0FBF2FAFFF765FD6043D9F8043045
:106A28009B00B0FBF3F3B3FBF8F308FB13A31B01C4
:106A38003233B3FBF8F303F00F033B433344AB604B
:106A4800BDE8F087FFF73EFD04FB00F3D9F80460CA
:106A58004FF06408B600B3FBF6F3B3FBF8F31E017E
:106A6800FFF730FD6043D9F804309B00B0FBF3F723
:106A7800FFF728FD6043D9F804309B00B0FBF3F31F
:106A8800B3FBF8F308FB13731B013233B3FBF8F3C2
:106A980003F0F007FFF716FD6043D9F804209200D1
:106AA800B0FBF2FAFFF70EFDB7E700BF0038014070
:106AB800F8B504460E4617461D4621680B6836EAA7
:106AC800030301D10020F8BD6B1CF7D095B92368EA
:106AD8000320DA6822F4D072DA605A6922F00102DF
:106AE8005A61202384F8393084F83A30002384F836
:106AF8003830F8BDFEF768FBC01B8542DDD2E6E7FB
:106B080010B5044640B390F8393003F0FF021BB9C2
:106B180080F8382001F0E2FC2423226884F8393018
:106B2800D368204623F40053D360FFF723FF23687C
:106B380000201A6922F490421A615A6922F02A0246
:106B48005A61DA6842F40052DA602023E06384F87C
:106B5800393084F83A3010BD012010BD2DE9F041DC
:106B68001F4690F839300446202B0D4690464ED1EA
:106B7800002949D0002A47D090F83830012B46D058
:106B8800012380F838300023C363212380F839308B
:106B9800FEF71AFB0646A4F82480A4F82680E38CA6
:106BA8009BB26BB93B46324640212046FFF780FF37
:106BB800A8B9202384F8380084F83930BDE8F0817A
:106BC800E38C3246013B9BB2E384A3688021B3F592
:106BD800805F20463B460ED1FFF76AFF10B10320C5
:106BE800BDE8F0812B882268C3F30803536023694A
:106BF80043B90235D3E7FFF75BFF0028EFD12368DD
:106C08002A785A600135CAE70120BDE8F0810220E0
:106C1800BDE8F08138B50446134694F83920202A97
:106C28002AD139B333B394F83820012A24D0012269
:106C3800002584F838202122E384206BE56384F85A
:106C480039200E4AA384216282620D4A4563C262DA
:106C58000C4A026322680432FEF710FE6FF040020D
:106C6800236828461A605A6984F8385042F080022E
:106C78005A6138BD012038BD022038BD236D000897
:106C8800516D00081D6E0008134690F83A2073B540
:106C9800202A054638D1002934D0002B32D090F86C
:106CA8003820012A30D00122002480F838202222FE
:106CB80081628385C46380F83A20406B134A2E684A
:106CC8008262134A4463C262124A02630A46311D51
:106CD800FEF7D4FD20462B6801941A6801925A6881
:106CE80085F838400192019ADA6842F48072DA60D5
:106CF8005A6942F001025A615A6942F040025A61E7
:106D080002B070BD0120FBE70220F9E75B6D0008C7
:106D1800116E00081D6E0008704708B50368426AC6
:106D28001B6813F020030AD1D38413685A6922F030
:106D380080025A61DA6842F04002DA6008BD104603
:106D4800FFF7EAFF08BD704708B5406AFFF7FBFF89
:106D580008BD08B50368426A1B6813F0200310D108
:106D6800D3851368D96821F48071D960596921F0F5
:106D780001015961596921F040015961202382F8C4
:106D88003A30104601F0E8FC08BD90F83A3010B5EA
:106D9800222B36D183680169B3F5805F0268836A64
:106DA80023D15268E9B9C2F3080223F8022B83629F
:106DB800C48D013CA4B2C4858CB90368DA6822F09A
:106DC8002002DA60DA6822F48072DA605A6922F006
:106DD80001025A61202380F83A3001F0BDFC0020FE
:106DE80010BDD2B223F8012BE1E721B9591C526832
:106DF80081621A70DCE75268591C816202F07F02D6
:106E0800F7E7022010BD704708B5406AFFF7FBFF9F
:106E180008BD7047416A08B50B685A6991F839008E
:106E280021280AD1120608D50022CA84DA6822F07D
:106E3800C002DA60202281F839205B6991F83A2093
:106E4800222A06D15B0604D500230846CB85FFF726
:106E580083FDCB6B084643F01003CB63FFF7D9FFE4
:106E680008BD0000036870B51A6804461607D9689B
:106E78005D6907D196065AD58D0658D5BDE870408C
:106E8800FFF783BF15F0010502D111F4907F4ED0B2
:106E9800D30705D5CE0542BFE36B43F00103E36397
:106EA800500704D51DB1E36B43F00203E363930776
:106EB80004D51DB1E36B43F00403E363160704D55F
:106EC8001DB1E36B43F00803E363E36B002B66D06B
:106ED800950604D5880602D52046FFF756FF236895
:106EE80020465D69E26B110702D415F040051AD0FF
:106EF800FFF732FD23685A69520610D55A69606B4C
:106F080022F040025A6150B1254B4363FEF7F4FC6E
:106F1800002844D0606BBDE87040436B184720469A
:106F2800FFF777FF70BDFFF774FFE56370BD1606C6
:106F380027D50D0625D594F83920212A2FD1A26806
:106F4800B2F5805F226A17D11188C1F30801596030
:106F5800216979B902322262E28C013A92B2E28462
:106F6800EAB9DA6822F08002DA60DA6842F04002B0
:106F7800DA6070BD0132EEE7511C216212785A6066
:106F8800EAE750060BD54A0609D5DA68204622F00A
:106F98004002DA60202384F83930FFF7BDFE70BD67
:106FA800AD6F000808B50023406AC385C384FFF7A6
:106FB80030FF08BD70B50022054604212448FEF7BD
:106FC800FDFF1024224E012208213046FEF7F6FF6D
:106FD8002B044CBF0122002210213046FEF7EEFFA1
:106FE800013C002208213046FEF7E8FF6D0014F04E
:106FF800FF04ADB2E7D101224FF400411548FEF776
:10700800DDFF0A2000F0D6FD22464FF4004111486A
:10701800FEF7D4FF012204210D48FEF7CFFF2246D8
:1070280010210B48FEF7CAFF01224FF4004109481E
:10703800FEF7C4FF224604210548FEF7BFFF22469B
:10704800BDE870404FF400410248FEF7B7BF00BFEB
:10705800002001400014014008B50120FEF7BAF8ED
:1070680048F20C00FFF7A6FF0120FEF7B3F84FF433
:107078002040FFF79FFFBDE808400120FEF7AAB8AF
:1070880084B02DE9F84F0AAC84E80F000E9EBDF8D5
:107098003C7000223946814630469DF84050BDF884
:1070A8002CA0DDF83080BDF834B0FEF787FF012052
:1070B800FEF790F8062415F0010218BF0122594680
:1070C8004046FEF77BFF012251464846FEF776FF11
:1070D8000120FEF77FF8002251464846FEF76EFF72
:1070E800013C0120FEF776F814F0FF044FEA55053D
:1070F800E1D1224651464846FEF760FF22464FF44A
:1071080080614046FEF75AFF0120FEF763F83946D2
:1071180001223046FEF752FF0120FEF75BF82246B7
:1071280039463046BDE8F84F04B0FEF747BF0000C7
:107138001FB50024424B029403F1100292E80300A9
:107148008DE803000FCBFFF79BFF3E4B029403F142
:10715800100292E803008DE803000FCBFFF790FFC1
:10716800394B029403F1100292E803008DE8030002
:107178000FCBFFF785FF354B029403F1100292E81D
:1071880003008DE803000FCBFFF77AFF304B029422
:1071980003F1100292E803008DE803000FCBFFF71C
:1071A8006FFF2C4B029403F1100292E803008DE864
:1071B80003000FCBFFF764FF274B029403F1100283
:1071C80092E803008DE803000FCBFFF759FF234B2C
:1071D800029403F1100292E803008DE803000FCB3C
:1071E800FFF74EFF1E4B029403F1100292E80300D2
:1071F8008DE803000FCBFFF743FF1A4B029403F10E
:10720800100292E803008DE803000FCBFFF738FF68
:10721800154B029403F1100292E803008DE8030075
:107228000FCBFFF72DFF114B029403F1100292E8E8
:1072380003008DE803000FCBFFF722FF04B010BD59
:107248000800002020000020380000205000002006
:10725800680000208000002098000020B000002076
:10726800C8000020E0000020F800002010010020E5
:1072780010B5FF230446221AD2B2914201D818460B
:1072880010BD14F8012B5340082213F0800F02F1AF
:10729800FF324FEA430318BF83F0310312F0FF02B5
:1072A800DBB2F2D1E7E730B5FF2305462C1AE4B28A
:1072B800A14203D89B1A5842584130BD15F8014BDA
:1072C8006340082413F0800F04F1FF344FEA4303AE
:1072D80018BF83F0310314F0FF04DBB2F2D1E5E705
:1072E80084B08DE80F009DF818209DF81C30029896
:1072F8001A4112F00102BDF80C1018BF012204B0A7
:10730800FEF75CBE84B02DE9F04F85B00EAC84E882
:107318000F00129DBDF84C60002231468046284679
:10732800BDF83C90FEF74AFE0A2000F043FC002717
:107338000DF1480B0DF1640A9DF85030FCB2029330
:107348001295ADF84C6003949BE803008DE80300A8
:10735800CDF83880ADF83C900EAB0FCBFFF7C0FFEF
:107368009DF86C30039402939AE803008DE80300BB
:1073780015AB0FCBFFF7B4FF9DF888300394029349
:1073880020AB93E803008DE803001CAB0FCBFFF79D
:10739800A7FF9DF8A4300394029327AB93E803005A
:1073A8008DE8030023AB0FCBFFF79AFF9DF8C030A1
:1073B800039402932EAB93E803008DE803002AABF5
:1073C8000FCBFFF78DFF9DF8DC300394029335ABAC
:1073D80093E803008DE8030031AB0FCBFFF780FF84
:1073E800012249464046FEF7E9FD0A2000F0E2FB8B
:1073F8000137002249464046FEF7E0FD082F9BD1A1
:1074080000224FF400410A48FEF7D8FD3146012218
:107418002846FEF7D3FD0A2000F0CCFB00223146B7
:10742800284605B0BDE8F04F04B0FEF7C7BD00BF61
:10743800000C0140F0B5274C274E25460FCE0FC54E
:1074480096E80300254F04F11C0685E803000FCFDA
:107458000FC697E80300224F86E803000FCF04F118
:1074680038060FC697E803001E4F86E803000FCFC3
:1074780004F154060FC697E803001B4F86E8030083
:107488000FCF04F170060FC697E80300174F86E880
:1074980003000FCF04F18C060FC697E80300002302
:1074A800A7B086E80300982229466846237684F820
:1074B800343084F8503084F86C3084F8883084F89C
:1074C800A43001F037FF94E80F00FFF71BFF27B047
:1074D800F0BD00BFD804002088010020580100201A
:1074E80028010020A0010020700100204001002098
:1074F80070B50223044601250020E60748BF05FAB7
:1075080003F603F1010348BF80190E2B4FEA540418
:10751800F3D10124CD0748BF04FA03F503F10103B1
:1075280048BF4019182B4FEA5101F3D1D30748BF80
:1075380000F1807070BDF0B50646012002240746B0
:107548009DF8145016F0010F18BF07FA04FE04F155
:10755800010418BF70440E2C4FEA5606F2D10126DA
:10756800CF0748BF06FA04F704F1010448BFC01961
:10757800122C4FEA5101F3D1D70744BF00F5802000
:107588001324DE0742BF012303FA04F40019EC07B1
:1075980048BF00F500209DF81830A90748BF00F53E
:1075A80080106A0748BF00F50010DB0748BF00F5E8
:1075B8008000F0BD000000002DE9F3470446B2FB4F
:1075C800F3F09A468846FCF781FF31A3D3E90023FC
:1075D800FCF7F2FF06460A980F46FCF777FF0246CB
:1075E8000B4630463946FDF711F92BA3D3E90023A2
:1075F800FCF7E2FFFDF7B8FA05460A2000FB08F0A1
:10760800FCF764FF002280468946254B3046394600
:10761800FDF7FCF802460B4640464946FDF7F6F8EA
:1076280000221F4BFDF7F2F800221D4BFDF7EEF884
:107638000F460646FDF798FA1FFA80F84046FCF711
:1076480045FF0B46024639463046FCF701FEFDF77A
:10765800ABFA06462846FDF7ADFB01463046FDF776
:1076680001FCFDF74FFD4146002280B2FFF740FFC5
:107678000023022206468DE80C0051460122A8B2DA
:10768800FFF759FF84E84100204602B0BDE8F087C3
:107698007B14AE47E17A843F0000000080842E41CD
:1076A80000408F400E4B9A7F4AB9DA7F3AB993F877
:1076B800202022B98722DA775F2283F8202093F8E6
:1076C80021205AB993F8222042B993F823202AB9E5
:1076D800992283F82220B12283F82320704700BF23
:1076E8008005002084B02DE9F04F85B00EAC84E809
:1076F8000F00179BBDF83C80C3F30A0ABDF8583049
:10770800109C0193159BBDF8445023F07F430293CE
:10771800149B129E23F07F43BDF84C700022414613
:1077280003938146FEF74AFC002229462046FEF7CD
:1077380045FC002239463046FEF740FC4FF00B0B63
:107748001AF4806218BF012229462046FEF736FC4B
:107758000A2000F02FFA012241464846FEF72EFC87
:107768000A2000F027FA002241464846FEF726FC88
:10777800BBF1010B4FEA4A0AE2D1012239463046F1
:10778800FEF71CFC0A2000F015FA5A463946304626
:10779800FEF714FC4FF0100A019B294613F400422F
:1077A80018BF01222046FEF709FC0A2000F002FA61
:1077B800012241464846FEF701FC0A2000F0FAF98A
:1077C800002241464846FEF7F9FB019BBAF1010A3F
:1077D8004FEA43039BB20193DED10122394630467A
:1077E800FEF7ECFB0A2000F0E5F952463946304630
:1077F800FEF7E4FB4FF0180A029B294613F4000237
:1078080018BF01222046FEF7D9FB0A2000F0D2F962
:10781800012241464846FEF7D1FB0A2000F0CAF98A
:10782800002241464846FEF7C9FB029BBAF1010A0D
:107838004FEA430323F07F430293DDD10122394607
:107848003046FEF7BBFB0A2000F0B4F95246394631
:107858003046FEF7B3FB4FF0180A039B294613F492
:10786800000218BF01222046FEF7A8FB0A2000F0FC
:10787800A1F9012241464846FEF7A0FB0A2000F084
:1078880099F9002241464846FEF798FB039BBAF156
:10789800010A4FEA430323F07F430393DDD15246A5
:1078A80029462046FEF78AFB394601223046FEF774
:1078B80085FB0A2000F07EF952463946304605B06D
:1078C800BDE8F04F04B0FEF779BB000038B50023DF
:1078D8001A4CBE2223601A4B0546A3600123E360BD
:1078E80043706023837061230270C370FEF776F9DA
:1078F80014492046FEF722FA18B1134802F002FA9A
:10790800FEE704462B195B782A5D04F1006102EB5F
:10791800032292B2002301F5FF210120FEF7A4F90A
:1079280020B1A521094802F079F9FEE70234642C58
:10793800E8D1BDE83840FEF763B900BF3C04002039
:1079480000F807084C04002058BC000866BC000872
:1079580008B5FFF7BBFF012008BD002303F1006253
:1079680002F5FF221188C1541288C1180233C2F3EC
:107978000722642B4A70F1D10120704770B5244D5D
:107988004FF480412846FEF713FB224C4FF4004188
:1079980084F843002846FEF70BFB1F4E84F844008A
:1079A80001213046FEF704FB022184F845003046E9
:1079B800FEF7FEFA802184F846001848FEF7F8FA28
:1079C80006F5006684F84A004FF400713046FEF769
:1079D800EFFA4FF4806184F849003046FEF7E8FA80
:1079E8004FF4006184F847003046FEF7E1FA4FF49F
:1079F800805184F848002846FEF7DAFA4FF480618F
:107A080084F84B002846FEF7D3FA84F84C0070BD82
:107A180000100140E3050020001801400014014057
:107A280043380A460D2840D8DFE800F0070D121841
:107A3800272C211C31363B3B3B3B01B101224FF443
:107A480080411B4808E001B101224FF40041F8E7EA
:107A580001B1012201211748FEF7B0BA01B1012294
:107A68000221F8E701B1012280211348F4E701B1AE
:107A780001224FF400711148EEE701B101224FF4E1
:107A88008061F8E701B101224FF40061F3E701B129
:107A980001224FF48051D4E701B101224FF48061F3
:107AA800CFE7064B11B1064A1A617047054AFBE752
:107AB800001001400018014000140140002001405E
:107AC800800160006000800110B5074CA178601C3F
:107AD800FFF7CEFB84F86100204601F08DFBBDE87E
:107AE800104000F06FBE00BF8005002070B52E4D1D
:107AF8002E4C284600228021FEF760FA20460022FC
:107B08004FF40071FEF75AFA204600224FF48061C4
:107B1800FEF754FA204600224FF40061FEF74EFAB1
:107B280028460022A5F580658021FEF747FA204EF9
:107B3800284600224FF48051FEF740FA28460022DA
:107B48004FF48061FEF73AFA304600220121FEF731
:107B580035FA304600220221FEF730FA2846002284
:107B68004FF48041FEF72AFA284600224FF40041DC
:107B7800FEF724FA204600222021FEF71FFA2046AD
:107B880000224021FEF71AFA204601228021FEF742
:107B980015FA204601224FF48071FEF70FFABDE86E
:107BA80070400120FDF716BB001401400020014081
:107BB80000180140084A0949126882B0B2FBF1F284
:107BC8000190019B53430193019B5A1E0192002B84
:107BD800FAD102B0704700BF1802002040420F00DF
:107BE80010B5064C2368B3F5FA7F06D94FF48041E7
:107BF8000348FEF7E8F90023236010BD580400206D
:107C08000020014040F6C4120B4BF0B519689142B0
:107C18001A460FD900231C46084F094E57F813007F
:107C280099190233050A1C2B81F8255081F8260082
:107C38001460F3D1F0BD00BF50040020A004002060
:107C4800E305002070B5074D074C084EAB68002BC4
:107C580002DD2368642B00D870BD304600F04CFD6F
:107C6800F4E700BFC40B00205C04002000070020DC
:107C780002680A4B9A420FD1094A1368013313600C
:107C8800084A136801331360074A13680133136005
:107C9800064A136801331360704700BF00100040A4
:107CA8005C040020580400205004002054040020E4
:107CB80010B514460A230248FEF750FF204610BDAF
:107CC8000007002010B596B0282200210CA801F06A
:107CD8003CFB1422002101A801F037FB18220021E7
:107CE8000DEB020001F031FB012310931023022455
:107CF80011934FF440130CA815930C941394FEF7AA
:107D080067F90F234FF4806201930023214601A8ED
:107D18000393049205930294FEF722FB4FF48043E9
:107D280006A806940893FEF7EDFB16B010BD0000F8
:107D380080B5B04D8CB0FDF729FAFFF7C3FF1022CC
:107D4800002108A801F001FBAB69002243F04003C1
:107D5800AB61AB697F2103F040030193019BAB69E1
:107D6800A54843F01003AB61AB69002403F010038E
:107D78000293029BAB69012643F08003AB61AB69B8
:107D8800022703F080030393039BAB694FF00C09B0
:107D980043F00403AB61AB694FF00E0803F0040332
:107DA8000493049BAB694FF0070A43F00803AB61E7
:107DB800AB6903F008030593059BAB6943F0200307
:107DC800AB61AB6903F020030693069BAB6943F4F0
:107DD8008073AB61AB6903F480730793079BFEF76D
:107DE800EDF800224FF6C0418448FEF7E7F800227C
:107DF80040F2F3318248FEF7E1F8002248F6FF71BD
:107E08008048FEF7DBF8002247F6FC717E48FEF753
:107E1800D5F800224FF400417C48FEF7CFF8002245
:107E280018217B48FEF7CAF87F2308A972480893EF
:107E380009960B970A94FDF7CFFF4FF6C04308A9A0
:107E48006E48089309960B970A94FDF7C5FF40F210
:107E5800F33308A96A48089309960B970A94FDF723
:107E6800BBFF08A96648CDF8209009940A94FDF74D
:107E7800B3FF48F6FF7308A96248089309960B9761
:107E88000A94FDF7A9FF4FF4405308A95D480893E9
:107E980009940A94FDF7A0FF47F6FC7308A95A480D
:107EA800089309960B970A94FDF796FF4FF44073D1
:107EB80008A95248089309940A94FDF78DFF4FF4D6
:107EC800004308A95148089309960B970A94FDF7AF
:107ED80083FF182308A94E48089309960B970A941C
:107EE800FDF77AFF602308A94948089309940A9482
:107EF800FDF772FF6B6933436B616B69454D334026
:107F08000093009B444B28462B604FF48073AB6072
:107F18004FF46023EE60EB61089409940A946C6155
:107F28006C60C5F81080FDF70FFB08A92846099674
:107F3800CDF828A00894FDF79BF90896032608A910
:107F480028460997FDF794F908A92846089709963D
:107F5800FDF78EF90896042608A928460996FDF724
:107F680087F90896052608A928460996FDF780F995
:107F78000896062608A928460996FDF779F908966D
:107F8800082608A92846CDF824A0FDF771F908A904
:107F98002846CDF820A00996FDF76AF90896092623
:107FA8004FF00A0A0B2708A928460996FDF760F939
:107FB80008960D2608A92846CDF824A0FDF758F9FB
:107FC80008A92846CDF820A00997FDF751F908A976
:107FD80028460897CDF82490FDF74AF908A92846BD
:107FE8000996CDF82090FDF743F908A92846089688
:107FF80014E000BF001002400018014000100140CA
:10800800001C01400014014000200140000801400C
:10801800000C01408C06002000240140CDF824808B
:10802800FDF726F94FF4E1334348444A846080E879
:108038000C00C4600461C0F814908461C461FEF748
:108048005FFD41F2DF533E4E3E49304686E80A0066
:1080580008940994B460C6F80CA0B461FEF73EFC1D
:1080680008A9304608940994FEF752FC2246214696
:108078002520FDF76DFB2520FDF79EFB22462146B6
:108088003620FDF765FB3620FDF796FB2246214694
:108098003846FDF75DFB3846FDF78EFB2246214644
:1080A8004046FDF755FB4046FDF786FB2246214634
:1080B8000F20FDF74DFB0F20FDF77EFB224800F057
:1080C800FBFA224B21461B68986801F023FEFFF754
:1080D8000DFDFFF753FC2846FDF7C0FA0028FAD13A
:1080E800FEF7BAFF1A48FFF738FCFFF7DBFA00F093
:1080F80043F8FFF79FF9FFF71BF8FFF7E5FC0E229F
:1081080014491548FDF770F9144801F0FBFD1448AF
:1081180001F0F8FD134A1449144801F07FFD144892
:1081280001F0F0FD0D4801F0EDFDFFF759FDFFF7F7
:1081380089FDFFF767FDF8E70007002000380140D8
:108148008407002000100040C40B00204C020020CF
:1081580080050020A00400208C06002077BC0008C1
:10816800A1BC0008AEBC0008B7BC0008C3BC00082E
:10817800D4BC000870470000104B9A7D2AB9DA7DFC
:108188001AB93E229A758022DA751A7E2AB95A7E61
:108198001AB938221A76D6225A769A7E2AB9DA7EFF
:1081A8001AB94D229A76EE22DA761A7F2AB95A7FC0
:1081B8001AB959221A77A6225A77704780050020E3
:1081C800012370B502241D46C60748BF05FA04F608
:1081D80004F1010448BF9B19082C4FEA5000F3D161
:1081E8000120CD0748BF00FA04F504F1010448BF97
:1081F8005B19152C4FEA5101F3D1D20748BF03F59B
:108208000013184670BD00004CF25033B0FBF3F376
:10821800372B09D905490022B0FBF1F1A3EB411036
:1082280080B289B2FFF7CCBF04207047006A1800FB
:1082380084B02DE9F74F0CAC84E80F00139BBDF810
:10824800347023F07F430193129BDDF83880BDF82A
:108258003C9023F07F43109DBDF8446000223946CE
:1082680000938246149CFDF7A9FE00224946404629
:10827800FDF7A4FE002231462846FDF79FFE4FF089
:10828800180B24F07F4414F4000218BF0122494659
:108298004046FDF793FE012239465046FDF78EFE13
:1082A8000A20FFF787FC002239465046FDF786FE74
:1082B8006400BBF1010B24F07F44E4D10122314674
:1082C8002846FDF77BFE0A20FFF774FC5A46314624
:1082D8002846FDF773FE1824009B494613F4000254
:1082E80018BF01224046FDF769FE01223946504673
:1082F800FDF764FE0A20FFF75DFC00223946504670
:10830800FDF75CFE009B013C4FEA430323F07F43EB
:108318000093E1D1012231462846FDF74FFE0A209D
:10832800FFF748FC224631462846FDF747FE182449
:10833800019B494613F4000218BF01224046FDF78D
:108348003DFE012239465046FDF738FE0A20FFF768
:1083580031FC002239465046FDF730FE019B013CB6
:108368004FEA430323F07F430193E1D131460122D1
:108378002846FDF723FE0A20FFF71CFC224631465B
:10838800284603B0BDE8F04F04B0FDF717BE000063
:108398000E4B82B09A6942F001029A619A6902F022
:1083A80001020092009ADA6942F08052DA61DB69D0
:1083B800074A03F080530193019B536823F0E0635D
:1083C80043F00073536002B0704700BF00100240D2
:1083D80000000140102230B5054689B00DEB0200BF
:1083E800002100F0B2FF2A682C4B9A4253D103F5C2
:1083F8006C439A69032442F400729A619A6904A949
:1084080002F400720092009A9A69254842F010021C
:108418009A619A6902F010020192019A9A6942F0EF
:1084280004029A619A6902F004020292029A9A6915
:1084380042F008029A619B69059403F008030393CC
:10844800039B0F230493FDF7C7FCFF2304A91548DA
:1084580004930594FDF7C0FC134804A904940594FB
:10846800FDF7BAFC8022114C114BE2604FF4007208
:1084780022614FF4006223606261002320222046BB
:108488006360A360A261E361FDF7B8F908B1FFF783
:1084980071FE2C62656209B030BD00BF0024014046
:1084A8000010014000080140000C01404007002076
:1084B800080002400268084B82B09A420AD103F5CC
:1084C8000033DA6942F01002DA61DB6903F0100365
:1084D8000193019B02B070470010004070B506463A
:1084E80086B01022002102A800F02FFF32682B4B23
:1084F8009A4251D103F558439A6902A942F480423D
:108508009A619A69264802F480420092009A9A6910
:10851800002542F004029A619B69224C03F004038F
:108528000193019B4FF400730293022303930323E7
:108538000593FDF751FC4FF48063194802A9029393
:1085480003950495FDF748FC174B204684E828005E
:108558008023A560E36025616561A561E561FDF79C
:108568004DF908B1FFF706FE4FF0100C0F4B74637E
:1085780066620F4C802284E8081000232046A3601E
:10858800E26023616361A361E361FDF737F908B134
:10859800FFF7F0FD3463666206B070BD0038014035
:1085A80000080140BC060020580002404400024078
:1085B800480600207047FEE7FEE7FEE7FEE7704743
:1085C80070477047FCF7F4BD0148FDF703BA00BFD8
:1085D800400700200148FDF7FDB900BF480600200C
:1085E8000148FDF7F7B900BFBC0600200148FEF7B7
:1085F80039BC00BF000700200148FEF781B800BF62
:108608008407002070B50E4615460C46A31B9D42F4
:1086180001DC284670BDAFF3008004F8010BF5E7D4
:1086280008B50A4B0246196809B90949196069462B
:10863800186802448A4206D900F052FE0C230360EF
:108648004FF0FF3008BD1A6008BD00BF600400206D
:10865800E41700204FF0FF3070474FF4005300201C
:108668004B60704701207047002070470E4B1A6816
:1086780042F001021A6059680C4A0A405A601A68A6
:1086880022F0847222F480321A601A6822F480225E
:108698001A605A6822F4FE025A604FF41F029A6068
:1086A800034A044B9A607047001002400000FFF82C
:1086B8000040000800ED00E00B4B10B51B680446B5
:1086C8000021986801F026FB0023084A63602360B4
:1086D800A3600749A2F800340648A2F80234BDE8AE
:1086E80010400122FEF7D0BA4C020020D00F002023
:1086F800D00B002000070020144A38B51068431C2E
:108708001360134B596803F10C040D5D114C0131D2
:10871800B1F5806F25541446A8BF00229D68B8BFE4
:10872800596005F1FF35A8BF5A609D606DB90948C9
:1087380000F062FD22682946064800F006FE256022
:108748000120BDE83840FCF745BD38BD6404002071
:10875800C40B0020C407002000230F4A10B5136083
:108768000E4C0F4A136022680132B2F5806FB8BF11
:1087780013462360A3680133B3F5806FA36001DB60
:10878800FFF7BAFF236807490122BDE810401944E2
:108798000548FEF779BA00BF5C040020C40B00202E
:1087A80050040020D00B00200007002008B5C37833
:1087B8008178C25C0130FEF776FD003018BF0120D9
:1087C80008BD0000BE2310B50B4C602123700223A6
:1087D80063706123601CA170E370FEF749FDEB2311
:1087E80084F8610084F862302146BDE810406322B5
:1087F8000248FEF70FBA00BFE3050020000700207B
:10880800BE2310B50A4C032123700423601C637037
:10881800A170E370FEF72CFDEB23A2782071637141
:108828002146BDE8104003320248FEF7F3B900BF05
:108838006804002000070020F0B5B54D02792B79B7
:10884800A9B0934204460CD0B24B029203F1100235
:1088580092E803008DE803000FCBFEF711FC2379A3
:108868002B7162796B7993420CD0AB4B029203F176
:10887800100292E803008DE803000FCBFEF700FC1E
:1088880063796B71A279AB7993420CD0A34B0292B6
:1088980003F1100292E803008DE803000FCBFEF706
:1088A800EFFBA379AB71E279EB7993420CD09C4B47
:1088B800029203F1100292E803008DE803000FCB47
:1088C800FEF7DEFBE379EB71227A2B7A93420CD028
:1088D800944B029203F1100292E803008DE8030022
:1088E8000FCBFEF7CDFB237A2B72627A6B7A934219
:1088F8000CD08D4B029203F1100292E803008DE830
:1089080003000FCBFEF7BCFB637A6B72A27AAB7ADB
:1089180093420CD0854B029203F1100292E80300B7
:108928008DE803000FCBFEF7ABFBA37AAB72E27ABC
:10893800EB7A93420CD07E4B029203F1100292E83C
:1089480003008DE803000FCBFEF79AFBE37AEB7286
:10895800227B2B7B93420CD0764B029203F11002C0
:1089680092E803008DE803000FCBFEF789FB237B19
:108978002B73627B6B7B93420CD06F4B029203F19B
:10898800100292E803008DE803000FCBFEF778FB96
:10899800637B6B73A27BAB7B93420CD0674B0292D9
:1089A80003F1100292E803008DE803000FCBFEF7F5
:1089B80067FBA37BAB73E27BEB7B93420CD0604BF2
:1089C800029203F1100292E803008DE803000FCB36
:1089D800FEF756FBE37BEB73237C2A7C9A4213D188
:1089E800697C627C91420FD1A97CA27C91420BD117
:1089F800E97CE27C914207D1297D227D914203D115
:108A0800697D627D914220D04E4E2B743376637C13
:108A180098226B7486F83430A37C06F11001AB748D
:108A280086F85030E37C6846EB7486F86C30237D1A
:108A38002B7586F88830637D6B7586F8A43000F056
:108A480079FC96E80F00FEF75DFCA37DAA7D9A42AB
:108A580003D1E97DE27D914235D0AB75E37DEB75BD
:108A6800A07DE37D43EA002337485843FFF7CCFB5A
:108A7800364A374B04924FF482620390029203F114
:108A8800100292E803008DE803000FCBFFF7D0FB3C
:108A98000120FCF79FFB22791E4B029203F1100282
:108AA80092E803008DE803000FCBFEF7E9FA1A4BB2
:108AB8006279029203F1100292E803008DE8030044
:108AC8000FCBFEF7DDFA237E2A7E607E9A4202D122
:108AD8006A7E824270D02B76687640EA03201A4B71
:108AE8005843FFF791FB194A1A4B04924FF48262DC
:108AF8000390029203F1100292E803008DE803004C
:108B08000FCBFFF795FB0120FCF764FB24E000BFC7
:108B1800E305002008000020200000203800002085
:108B280050000020680000208000002098000020ED
:108B3800B0000020C8000020E0000020F80000205D
:108B480010010020D8040020A086010092809F0018
:108B5800B8010020D0010020A279C54B029203F190
:108B6800100292E803008DE803000FCBFEF788FAA5
:108B7800E279C04B029203F1100292E803008DE8FB
:108B880003000FCBFEF77CFA227ABB4B029203F16B
:108B9800100292E803008DE803000FCBFEF770FA8D
:108BA800B64B627A029203F1100292E803008DE854
:108BB80003000FCBFEF764FAA37EAA7EE07E9A42FA
:108BC80002D1EA7E824232D0AB76E87640EA0320D0
:108BD800AB4B5843FFF718FBAA4AAB4B04924FF430
:108BE80082620390029203F1100292E803008DE87A
:108BF80003000FCBFFF71CFB0120FCF7EBFAA27A6E
:108C0800A24B029203F1100292E803008DE80300E0
:108C18000FCBFEF735FA9E4BE27A029203F110026F
:108C280092E803008DE803000FCBFEF729FA237FB3
:108C38002A7F9A4203D1697F627F91424DD02B7778
:108C4800637F6B77207F637F43EA00238C48584318
:108C5800FFF7DAFA8B4A8F4B04924FF48262039043
:108C6800029203F1100292E803008DE803000FCB93
:108C7800FFF7DEFA0120FCF7ADFA227B864B029261
:108C880003F1100292E803008DE803000FCBFEF712
:108C9800F7F9627B814B029203F1100292E803001C
:108CA8008DE803000FCBFEF7EBF9A27B7C4B029219
:108CB80003F1100292E803008DE803000FCBFEF7E2
:108CC800DFF9784BE27B029203F1100292E803008D
:108CD8008DE803000FCBFEF7D3F9A37FAA7F9A4252
:108CE80009D1E97FE27F914205D195F8201094F8E7
:108CF800202091422AD0AB77E37F4FF44052EB77A4
:108D080094F8203085F82030E17FA37F090241EAFA
:108D1800034141F2883394F820000093014308236B
:108D280026A8FEF749FC0322059241F2C2420492AA
:108D3800269A5D4B0392279A029203F1100292E859
:108D480003008DE803000FCBFEF7CCFC94F821302C
:108D580095F821209A420BD195F8221094F82220F8
:108D6800914205D195F8231094F8232091422FD0F1
:108D780085F8213094F822304FF4405285F822309B
:108D880094F8233085F8233094F8221094F8213091
:108D9800090241EA034141F2883394F82300009321
:108DA8000143082326A8FEF707FC0322059241F297
:108DB800C2420492269A3D4B0392279A029203F1EB
:108DC800100292E803008DE803000FCBFEF78AFC3F
:108DD80094F8431095F843308B4206D04320FEF7B1
:108DE8001FFE94F8433085F8433094F8441095F802
:108DF80044308B4206D04420FEF712FE94F84430EB
:108E080085F8443094F8451095F845308B4206D0E3
:108E18004520FEF705FE94F8453085F8453094F86E
:108E2800461095F846308B4206D04620FEF7F8FDEE
:108E380094F8463085F8463094F84A1095F84A3048
:108E48008B4206D04A20FEF7EBFD94F84A3085F8AD
:108E58004A3094F8491095F849308B4228D0492077
:108E6800FEF7DEFD94F8493085F8493020E000BF70
:108E780038000020500000206800002080000020FA
:108E8800A086010092809F00E80100209800002041
:108E9800B000002000020020C8000020E0000020F0
:108EA800F800002010010020340200201C020020DD
:108EB80094F8471095F847308B4200F090810126CE
:108EC8004720FEF7ADFD94F8473085F8473094F811
:108ED800481095F848308B4207D001264820FEF705
:108EE8009FFD94F8483085F8483094F84B1095F871
:108EF8004B308B422DD04B20FEF792FD94F84B302F
:108F0800012085F84B30FCF765F994F84B3003B332
:108F180095F8221095F82130090241EA034195F8A5
:108F2800233042F21070194341F28833AF4F414366
:108F380000934FF44052082326A8FEF73DFB9822E1
:108F480007F11001684600F0F5F997E80F00FEF701
:108F5800D9F994F84C1095F84C308B422AD04C2013
:108F6800FEF75EFD94F84C30012085F84C30FCF794
:108F780031F994F84C30EBB1E97FAB7F090241EA53
:108F8800034195F8203042F21070194341F28833BA
:108F9800964F41430093964A022326A8FEF70CFBFE
:108FA800982207F11001684600F0C4F997E80F000D
:108FB800FEF7A8F994F84D3095F84D209A4206D05E
:108FC80085F84D3094F84D104D20FEF729FD94F8A2
:108FD8004E3095F84E209A4206D085F84E3094F8D7
:108FE8004E104E20FEF71CFD824D94F84F3095F838
:108FF8004F209A4206D085F84F3094F84F104F20F2
:10900800FEF70EFD94F8503095F850209A4206D09D
:1090180085F8503094F850105020FEF701FD94F870
:10902800513095F851209A4205D195F8521094F88C
:109038005220914206D0012685F8513094F85230DA
:1090480085F8523094F8533095F853209A4205D158
:1090580095F8541094F85420914207D085F853306D
:1090680094F8543046F0020685F8543094F8553098
:1090780095F855209A4205D195F8561094F856203F
:10908800914207D085F8553094F8563046F00406DA
:1090980085F8563094F8573095F857209A4205D1FC
:1090A80095F8581094F85820914207D085F8573011
:1090B80094F8583046F0080685F8583094F8593036
:1090C80095F859209A4205D195F85A1094F85A20E3
:1090D800914207D085F8593094F85A3046F0100676
:1090E80085F85A3094F85B3095F85B209A4205D1A0
:1090F80095F85C1094F85C20914207D085F85B30B5
:1091080094F85C3046F0200685F85C3094F85D30C1
:1091180095F85D209A4205D195F85E1094F85E2086
:10912800914207D085F85D3094F85E3046F04006ED
:1091380085F85E3094F85F3095F85F209A4205D143
:1091480095F8601094F8602091424AD085F85F3015
:1091580094F8603085F8603095F8523095F85100F1
:1091680043EA0020FDF726FF95F8543095F85300A0
:1091780043EA0020FDF71EFF95F8563095F8550094
:1091880043EA0020FDF716FF95F8583095F8570088
:1091980043EA0020FDF70EFF95F85A3095F859007C
:1091A80043EA0020FDF706FF95F85C3095F85B0070
:1091B80043EA0020FDF7FEFE95F85E3095F85D0065
:1091C80043EA0020FDF7F6FE95F85F0095F8603059
:1091D80043EA002029B0BDE8F040FDF7EBBE0026C9
:1091E80075E6002EB8D129B0F0BD00BFD804002024
:1091F800005A6202E305002070B504464678FFF77E
:10920800D5FA054648B9A27840F6B8330332214664
:109218001A48FDF7A3FC284670BD032EFBD8DFE8EB
:1092280006F0022026290023154EA2785D1C05327F
:10923800DBB29A420FDA134800F064FDBFF34F8F98
:109248001149124BCA6802F4E0621343CB60BFF3C2
:109258004F8F00BFFDE7E15C304600F0DFFC2B4696
:10926800E3E72046FFF7E8FAFFF7CAFAD3E7FFF784
:10927800A9FAD0E70648FEF76BFBF5E700070020E0
:109288000ABD000810BD000800ED00E00400FA0562
:10929800E3050020002103E00B4B5B5843500431E9
:1092A8000A480B4B42189A42F6D30A4A02E00023B6
:1092B80042F8043B084B9A42F9D3FFF7D7F900F07C
:1092C80015F8FEF735FD7047E8BF000800000020DC
:1092D8001C04002020040020E4170020FEE7000002
:1092E800014B1868704700BF4C02002070B500257C
:1092F8000C4E0D4CA41BA410A54209D102F08AFC07
:1093080000250A4E0A4CA41BA410A54205D170BD25
:1093180056F8253098470135EEE756F82530984736
:109328000135F2E7E0BF0008E0BF0008E0BF000831
:10933800E4BF000810B5431E0A44914200D110BD95
:1093480011F8014B03F8014FF7E703460244934233
:1093580000D1704703F8011BF9E7002B2DE9F0470E
:109368001E46BBBF03F100431E4600232D2388B0D1
:10937800149F129927F02007462F1446109DDDF8F8
:109388004CA00B7004D0452F00D10135022300E01A
:10939800032307AA049206AA03928DE8280422460A
:1093A800334600F0B9FE472F804602D1119BDB07F8
:1093B80026D5462F08EB050911D198F80030302B37
:1093C8000AD10022002320463146FBF75DFB18B97D
:1093D800C5F10105CAF80050DAF8003099440022B6
:1093E800002320463146FBF74FFB38B93022079B54
:1093F800994505D9591C07911A70F8E7CDF81C90C2
:109408004046079B159AA3EB0803136008B0BDE814
:10941800F0870346F7B5002903F8022BB6BF2D22C3
:109428002B2249420929427021DD0DF10702174616
:109438000A2691FBF6F506FB1511092D01F13001FD
:1094480002F8011C02F1FF34294609DC3031023AE6
:1094580004F8011CBA421C4604D3201A03B0F0BD1C
:109468002246E6E712F8011B03F8011BF2E7302257
:109478001C46114404F8022B5970EEE72DE9F04F11
:1094880091B00C461A9F93461E46054601F094FD7E
:10949800036818460993FAF7C3FE00230E933B6846
:1094A8000A90073323F0070303F1080294F81880A1
:1094B800D4F800A03A60D3E90023C4E91223D4F811
:1094C8004C90A76C29F000430B934FF0FF32A64B4A
:1094D80038460B99FBF70AFB002840F0F7814FF05C
:1094E800FF32A14B38460B99FBF7E2FA002840F00F
:1094F800ED810022002338464946FBF7CFFA10B128
:109508002D2384F84330994B994FB8F1470F98BFF2
:109518001F4603234FF0000923612AF00403236048
:1095280000965B460FAA2146284600F0DFF9013075
:1095380040F09A804FF0FF3011B0BDE8F08F6268BC
:109548000EA8531C0DF1340E4AF4806341D1062253
:10955800626000212360019363680DF13302059076
:10956800029200933A464B460691CDF81080CDF80A
:109578000CE02846FFF7F1FE08F0DF03472B07460B
:1095880009D10D9BD81C02DB6268934259DDA8F112
:1095980002085FFA88F8B8F1650F0D9936D80139D5
:1095A800424604F150000D91FFF733FF0E9A8146B1
:1095B8008318012A236102DC2268D10701D501330F
:1095C80023619DF83330002BAAD02D2384F8433033
:1095D800A6E7B8F1670F02D0B8F1470FB9D19AB131
:1095E800002106910DF133018DE80C0023600590F0
:1095F8003A46CDF81080CDF80CE002914B4628464B
:10960800FFF7ABFE0746BCE70122A1E7B8F1660FFA
:1096180019D1002963680CDD216113B92268D207CA
:1096280002D501330B4423610D9B4FF00009A3655C
:10963800C7E713B92268D00701D50233F3E701233E
:10964800F1E74FF067080D9B0E9A934205DB2268FD
:109658002361D107E8D50133E5E7002BCCBF01230F
:10966800C3F102031344DEE723685A0507D42369CC
:109678003A4659462846B04701302AD15AE7B8F148
:10968800650F40F2DC80D4E9120100220023FBF7C9
:10969800FBF9002839D00123364A59462846B047F5
:1096A80001303FF447AF0E9B0D9A9A4202DB2368C4
:1096B800D8070ED50A9B099A59462846B047013063
:1096C8003FF438AF002704F11A080E9B013B9F4274
:1096D80011DB23689F0708D5002704F11908E36800
:1096E8000F9A9B1A9F42C0F2E780E0680F9B98424E
:1096F800B8BF184620E70123424659462846B047D6
:1097080001303FF417AF0137DFE70D9B002B33DC47
:109718000123184A59462846B04701303FF40AAF9A
:109728000D9B23B90E9B13B92368D907D1D50A9B82
:10973800099A59462846B04701303FF4FBAE4FF02E
:10974800000804F11A090D9B5B42984501DB0E9B4A
:109758008EE701234A4659462846B04701303FF470
:10976800E9AE08F10108EEE7FFFFEF7F24BD00082E
:1097780028BD0008C1BC00080E9AA36D9A42A8BF74
:109788001A46002A904636DC4FF0000A04F11A0304
:1097980028EAE8780B93D4F85890A9EB08039A457F
:1097A80031DB0E9B0D9A9A4238DB2368DA0735D4F1
:1097B8000E9B0D99A3EB0902A3EB01089045A8BFE6
:1097C8009046B8F1000F31DC002728EAE87804F168
:1097D8001A090D9A0E9B9B1AA3EB08039F42BFF62A
:1097E80078AF01234A4659462846B04701303FF42E
:1097F800A1AE0137EDE7134659463A462846B04729
:109808000130C1D196E601230B9A59462846B04744
:1098180001303FF48FAE0AF1010ABCE70A9B099AAE
:1098280059462846B0470130C2D183E6434607EB84
:10983800090259462846B0470130C5D17AE60E9A42
:10984800012A01DCDB0734D501233A46594628466C
:10985800B04701303FF46EAE0A9B099A5946284634
:10986800B04701303FF466AED4E91201002200236C
:10987800FBF70AF950B1002704F11A080E9B013BC7
:109888009F420CDB4B4604F15002F2E60E9B7A1C19
:10989800013B59462846B0470130F3D14AE6012337
:1098A800424659462846B04701303FF443AE013797
:1098B800E4E701233A46ECE70123424659462846A5
:1098C800B04701303FF436AE013708E73A464B4619
:1098D80038464946FBF70AF900283FF430AE014BF9
:1098E800014F12E62CBD000830BD00082DE9F047F5
:1098F80091461F468A680B6906469342B8BF1346CD
:10990800C9F8003091F843200C46DDF8208012B1E8
:109918000133C9F800302368990642BFD9F80030EE
:109928000233C9F80030256815F0060507D104F19F
:10993800190AE368D9F800209B1A9D422ADB94F89B
:1099480043302268003318BF012392062FD404F154
:10995800430239463046C047013022D02368E568C3
:1099680003F00603042B18BF0025D9F800204FF098
:10997800000908BFAD1AA368226908BF25EAE57582
:109988009342C4BF9B1AED181A344D451BD10020D1
:10999800BDE8F0870123524639463046C0470130BA
:1099A80003D14FF0FF30BDE8F0870135C1E7302023
:1099B800E11881F843005A1C94F8451022440233F8
:1099C80082F84310C3E70123224639463046C04790
:1099D8000130E6D009F10109D7E700002DE9F0438D
:1099E80017460A7E85B06E2A984606460C460C9B9A
:1099F80001F1430E00F0BC801AD8632A2ED00AD891
:109A0800002A00F0C880582A00F08A8004F1420534
:109A180084F842202AE0642A01D0692AF6D1216814
:109A28001A6811F0800F23D0111D1960136827E000
:109A3800732A00F0B48008D86F2A2AD0702AE5D19A
:109A48000A6842F020020A6003E0752A21D0782AC9
:109A5800DCD178226F4984F8452064E01A6801F166
:109A68004205111D1960136884F842300123A3E0F0
:109A780011F0400F02F104011960D7D0B2F900309B
:109A8800002B03DA2D225B4284F8432062490A2224
:109A980017E02068196810F0800F03D0081D1860BF
:109AA8000B6806E010F0400F01F104001860F7D0D1
:109AB8000B886F2A14BF0A2208225749002084F80D
:109AC80043006568002DA560C0F29C80206820F0E6
:109AD80004002060002B3FD1002D40F09580754692
:109AE800082A0BD12368DA0708D5236962689A42E5
:109AF800DEBF302305F8013C05F1FF35AEEB050369
:109B08002361CDF800803B4603AA21463046FFF783
:109B1800EDFE013055D14FF0FF3005B0BDE8F083C0
:109B280081F845203C492268186812F0800F00F13E
:109B380004051D6001D0036802E05506FBD50388C3
:109B4800D00744BF42F0200222601BB9226822F0ED
:109B5800200222601022B1E77546B3FBF2F002FB47
:109B68001033CB5C05F8013D03460028F5D1B7E773
:109B780008681A6810F0800F496904D0101D186031
:109B88001368196007E010F0400F02F10400186034
:109B98001368F6D01980002375462361B1E71A6867
:109BA800111D1960156800216268284601F07EFAC7
:109BB80008B1401B606063682361002384F8433068
:109BC8009FE723692A4639463046C0470130A2D06C
:109BD80023689B0707D5002504F11909E368039A50
:109BE8009B1A9D4205DBE068039B9842B8BF184664
:109BF80093E701234A4639463046C04701308AD0A8
:109C08000135EBE7002BA7D10B7804F1420584F866
:109C1800423065E745BD000834BD00080FB40A4B63
:109C280013B51C6824B1A36913B9204601F03AF9A9
:109C380005AB049AA1682046019301F0F7FD02B034
:109C4800BDE8104004B070474C02002070B50E46C5
:109C5800054618B183690BB901F024F9AB69AC6802
:109C680013B9284601F01EF9234B9C4217D16C68A2
:109C7800A3891B071DD52369DBB1013EA36816F82C
:109C8800011F013BA360E9B9002B2EDA22460A2105
:109C9800284600F0F5F8013011D00A2070BD174BA6
:109CA8009C4201D1AC68E3E7154B9C4208BFEC68C5
:109CB800DEE72146284600F035F90028DDD04FF0D0
:109CC800FF3070BD002B04DAA269934206DB0A2933
:109CD80004D023685A1C22601970CFE72246284610
:109CE80000F0CEF80130C9D1E9E70A2023685A1CF0
:109CF8002260187070BD00BF84BD0008A4BD0008B4
:109D080064BD0008024B01461868FFF79FBF00BFFB
:109D18004C02002000294FF480630CBF022200226D
:109D280000F000B82DE9F7431D46514B04461E6864
:109D38000F46904626B1B36913B9304601F0B2F820
:109D48004C4B9C4252D17468B8F1020F06D0B8F15E
:109D5800010F00F28980002DC0F28680214630462E
:109D680001F036F8616B41B104F14403994202D025
:109D7800304601F089FC002363630023A36163601C
:109D8800A3891B0603D52169304601F07DFCA38910
:109D9800B8F1020F23F44A6323F00303A3815DD0D3
:109DA80001AB6A462146304601F014F9A3891843ED
:109DB800A0812DBB009D284601F070F907460028B8
:109DC8004ED1DDF80090A9453CD14FF0FF30A38972
:109DD80043F00203A3810023A36004F14703236037
:109DE80023610123636103B0BDE8F083224B9C42E9
:109DF80001D1B468A8E7214B9C4208BFF468A3E7E7
:109E0800002FD8D0B36913B9304601F04BF8B8F138
:109E1800010F08BFA389276004BF43F00103A38192
:109E2800A389276113F0080065611BD013F00100B6
:109E38004FF000031FBF6D42A360A561184608BF1D
:109E4800A560D0E7484601F029F907460028BCD0AC
:109E5800A3894D4643F08003A381D3E70020B6E7EA
:109E6800A946F5E7A060BEE74FF0FF30BBE700BFAB
:109E78004C02002084BD0008A4BD000864BD000891
:109E8800F8B50E461446054618B183690BB901F0BA
:109E980009F8214B9C422AD16C68A369A360A38965
:109EA8001A072ED5236963B323692068F6B2C01A4E
:109EB80063693746984204DB2146284600F088FF4C
:109EC80028BBA3680130013BA36023685A1C2260A9
:109ED8001E706369984204D0A389DB0719D50A2E3E
:109EE80017D12146284600F073FF90B10FE00B4BC5
:109EF8009C4201D1AC68D0E7094B9C4208BFEC6892
:109F0800CBE72146284600F00DF80028CCD04FF0CA
:109F1800FF373846F8BD00BF84BD0008A4BD00085F
:109F280064BD0008324B70B51D6806460C4625B165
:109F3800AB6913B9284600F0B5FF2E4B9C420FD1F0
:109F48006C68B4F90C309AB215072CD4D00611D429
:109F58000922326043F04003A3814FF0FF3070BD07
:109F6800254B9C4201D1AC68EBE7244B9C4208BFCF
:109F7800EC68E6E7510712D5616B41B104F144037F
:109F8800994202D0304601F07FFB00236363A38926
:109F980023F02403A3810023636023692360A3893A
:109FA80043F00803A38123694BB9A38903F4207301
:109FB800B3F5007F03D02146304601F02FF8A2897F
:109FC80012F001030CD00023A36063695B42A36114
:109FD800236953B9B4F90C3013F08000BAD170BDBD
:109FE800920758BF6369A360F2E70020F7E700BF54
:109FF8004C02002084BD0008A4BD000864BD000810
:10A008002DE9F74F03690C6980469C4200F3828072
:10A01800013C01F1140700F1140657F8245056F8D2
:10A0280024000135B0FBF5F54FEA840E06EB0E036C
:10A0380007EB0E0901938DB34FF0000A3846B4467A
:10A04800D34650F8042B93B205FB03A3120C4FEA36
:10A05800134A05FB02A29BB2ABEB0303BCF800B0AA
:10A068004FEA124A5B441FFA82FBDCF80020814564
:10A07800CBEB124202EB23429BB243EA02434FEA84
:10A08800224B4CF8043BDCD256F80E3033B9019B16
:10A09800043B9E421A4631D3C8F81040404601F0AE
:10A0A8001CFA002826DB30464FF0000E013557F821
:10A0B800041BD0F800C08BB2AEEB03031FFA8CF27E
:10A0C80013440A0CC2EB1C4202EB23429BB243EA44
:10A0D8000243B9454FEA224E40F8043BE7D256F80E
:10A0E800242006EB84032AB9043B9E421A460BD36C
:10A0F800C8F81040284603B0BDE8F08F1268043B4A
:10A10800002AC9D1013CC4E71268043B002AEFD1F8
:10A11800013CEAE70020EEE72DE9F04F466A95B0EA
:10A128000446219DCDE902233EB9102000F0B6FF78
:10A138006062466086600660C660636A196851B1ED
:10A148005A68012393404A608B60204600F0F0FF74
:10A158000022636A1A60039B002BB7BF0123002308
:10A168002B60039BAEBF2B6023F000430393DDF805
:10A178000C90AB4B33EA09031BD142F20F73209AC0
:10A188001360029B23B9C9F31300002800F08385EC
:10A19800229B53B9A34B21E0A34B06930833229A81
:10A1A8001360069815B0BDE8F08F9E4B06930333F5
:10A1B800F5E7DDE902670022002330463946FAF761
:10A1C80063FC804660B10123209A1360229B002B18
:10A1D80000F05E85954B229A1360013B0693E0E7F9
:10A1E80012AB019313AB009332463B46204601F075
:10A1F800EDF9C9F30A558246002D7DD03046C7F3E4
:10A20800130343F07F5141F44011A5F2FF35CDF817
:10A2180040800022864BFAF71BF87BA3D3E9002382
:10A22800FAF7CAF97AA3D3E90023FAF713F806462E
:10A2380028460F46FAF75AF977A3D3E90023FAF725
:10A24800BBF902460B4630463946FAF703F806468C
:10A258000F46FAF761FC0022834600233046394650
:10A26800FAF71CFC58B15846FAF740F902460B4673
:10A2780030463946FAF708FC08B90BF1FF3BBBF149
:10A28800160F58D8DDE902236A4901EBCB01D1E961
:10A298000001FAF721FC00284FD000230BF1FF3B07
:10A2A8000D93129B5D1B6B1E079343BF0023C5F1E3
:10A2B800010807934FF00008BBF1000F3FDB079B35
:10A2C800CDF830B05B440793002308931E9B092BFD
:10A2D80000F2B480052BC4BF043B1E931E9BC8BF6D
:10A2E8000026A3F10203D8BF0126032B00F2B28097
:10A2F800DFE803F084862D78139B129D1D4405F238
:10A308003243202B11DD029A05F21240C3F14003BB
:10A3180022FA00F009FA03F31843FAF7D7F80123F1
:10A32800A1F1F871013D109373E7C3F12000029B7E
:10A3380003FA00F0F1E70123B2E70D90B1E7CBF1A2
:10A34800000308930023A8EB0B080C93BEE7012336
:10A3580009931F9B002B40F38080994604930022A9
:10A368000421656A6A6001F114029A427AD969681F
:10A37800204600F0A9FE636A28601B68B9F10E0F39
:10A38800069300F2F080002E00F0ED80DDE9022354
:10A39800BBF1000FCDE90E2379DD264A0BF00F0340
:10A3A8004FEA2B1602EBC303F006D3E90023CDE9ED
:10A3B8000A235CD5DDE90E011F4B0325D3E90823E9
:10A3C800FAF724FACDE9020106F00F061A4F002E1B
:10A3D8004FD1DDE90A23DDE90201FAF717FACDE9E1
:10A3E80002016EE0012309931F9B5B4403F10109FD
:10A3F80004934B46012BB8BF0123B0E70023A7E71E
:10A408000023F0E7AFF3008061436F63A787D23F73
:10A41800B3C8608B288AC63FFB799F501344D33F4B
:10A428000000F07F5FBD000856BD0008C2BC0008F0
:10A438000000F83FF0BD0008C8BD00080126002351
:10A4480009961E934FF0FF33002204939946122376
:10A458001F9284E701230993F4E7012304939946A3
:10A468001A46F5E76A68490001326A607BE7022507
:10A47800ACE7F10708D5DDE90A01D7E90023FAF7C7
:10A488009BF8CDE90A010135761008379FE700F0FF
:10A49800A580DDE90E01CBF10006A24B06F00F0204
:10A4A80003EBC203D3E90023FAF786F80225002359
:10A4B800CDE902019C4F3611002E40F08480002B1C
:10A4C8008DD10D9B002B00F08B80DDE90223CDE9B7
:10A4D8000A23DDE90A010022944BFAF7DFFA002883
:10A4E8007ED0B9F1000F7BD0049B002B37DDDDE96E
:10A4F8000A0100228E4BFAF75FF8CDE90201049EAB
:10A508000BF1FF3701352846F9F7F0FFDDE90223A3
:10A51800FAF752F8874B0022F9F79CFECDE90A01B9
:10A528000B9BA3F150750B95002E5CD1DDE9020160
:10A538000022814BF9F78CFE0A9A2B46CDE90201DD
:10A54800FAF7CAFA002840F0F782DDE902010A9A10
:10A5580005F10043FAF7A2FA002840F0EB82DDE9A2
:10A568000E23CDE90223139B002BC0F25081BBF1CF
:10A578000E0F00F34C816B4B03EBCB03D3E90023A5
:10A58800CDE904231F9B002B80F2DA80B9F1000F7C
:10A5980000F3D68040F0CD82DDE904010022664B4D
:10A5A800FAF70AF8DDE90223FAF78CFA4E464F4625
:10A5B800002840F0A482069B069A5D1C31230BF10B
:10A5C800010B13709FE2F20705D5D7E90023F9F7CD
:10A5D800F3FF01230135761008376DE7022570E790
:10A5E8005F464E468FE7069A4E4B32441192099ABF
:10A5F800711E002A48D003EBC103D3E900230020D1
:10A608004E49FAF703F9DDE90A23F9F721FECDE906
:10A618000A01069DDDE90201FAF77EFA0646F9F716
:10A6280065FF02460B46DDE90201F9F711FEDDE997
:10A638000A23303605F8016BCDE90201FAF72EFA44
:10A64800002864D1DDE9022300203849F9F700FE2B
:10A65800DDE90A23FAF722FA002840F0B980119BB5
:10A668009D423FF47CAFDDE90A010022304BF9F747
:10A67800A3FF0022CDE90A01DDE902012C4BF9F71D
:10A688009BFFCDE90201C5E703EBC101D1E9000158
:10A69800DDE90A23F9F790FFCDE90A01069DDDE916
:10A6A8000201FAF739FA0646F9F720FF02460B4687
:10A6B800DDE90201F9F7CCFD3036119B05F8016B95
:10A6C800AB42CDE902014FF0000224D11B4BDDE97A
:10A6D8000A01F9F7BFFD02460B46DDE90201FAF768
:10A6E800FBF9002874D1DDE90A2300201349F9F7A2
:10A6F800AFFD02460B46DDE90201FAF7CFF9002863
:10A708003FF42DAF15F8013C6A1E302B01D0BB4633
:10A718004DE01546F6E7064BF9F74EFFCDE9020185
:10A72800BDE700BFF0BD0008C8BD00080000F03F4D
:10A738000000244000001C40000014400000E03FDE
:10A74800069DDDE90267DDE9042330463946FAF75C
:10A758005DF8FAF7E1F98046F9F7C8FEDDE9042368
:10A76800F9F72AFF02460B4630463946F9F770FDDD
:10A7780008F1300605F8016B069E0246AE1BB1458E
:10A788000B4637D1F9F766FD06460F4602460B46DB
:10A79800DDE90401FAF782F9C8B9DDE904013246B6
:10A7A8003B46FAF771F910B118F0010F0FD1514675
:10A7B800204600F0BDFC0023209A2B700BF101030A
:10A7C8001360229B002B3FF4ECAC1D60E9E45F466C
:10A7D80015F8012C6B1E392A06D1069A9A4207D120
:10A7E80030231370134601371A7801321A708EE736
:10A7F8001D46EDE70022B54BF9F7DEFE00220023E7
:10A8080006460F46FAF740F900289CD0CFE7099A88
:10A81800002A00F029811E9A012A00F30E81109A5D
:10A82800002A00F0068103F233434546089E079A42
:10A8380001211A4420469844079200F019FD074662
:10A84800002D0BDD079B002B08DDAB42A8BF2B4674
:10A85800079AA8EB0308ED1AD31A0793089BFBB1D4
:10A86800099B002B00F00481002E11DD3946324689
:10A87800204600F093FD524601460746204600F068
:10A8880000FD51460A90204600F052FC0A9B9A4669
:10A89800089B9A1B04D05146204600F07FFD824653
:10A8A8000121204600F0E4FC0C9B0646002B40F3F7
:10A8B800E1801A460146204600F070FD1E9B0646C0
:10A8C800012B40F3DA8000230893336906EB8303F6
:10A8D800186900F07FFCC0F12000079B184410F0B5
:10A8E8001F0000F0F080C0F12003042B40F3E28049
:10A8F800079BC0F11C008044054403440793B8F14A
:10A90800000F05DD51464246204600F095FD82467F
:10A91800079B002B05DD31461A46204600F08CFDCA
:10A9280006460D9B002B00F0D3803146504600F0C0
:10A93800D4FD002880F2CC80002351460A2220460C
:10A9480000F00DFC099B0BF1FF3B8246002B00F049
:10A95800A981002339460A22204600F000FC049B06
:10A968000746002B03DC1E9B022B00F3B980002D49
:10A9780005DD39462A46204600F05EFD0746089B5D
:10A98800002B00F010817968204600F09DFB0546F9
:10A998003A6907F10C01023292000C30FEF7CAFC4A
:10A9A80001222946204600F047FD07970746029BEB
:10A9B800DDF8188003F00103089331465046FFF78D
:10A9C8001FFB0799054600F13009504600F085FD48
:10A9D8003A4602903146204600F099FDC368024687
:10A9E800002B40F0E28001460990504600F075FDCA
:10A9F8000346099A11462046099300F099FB099BE2
:10AA0800002B40F0D4801E9A002A40F0D080089A8B
:10AA1800002A40F0CC80B9F1390F00F0E880029BA1
:10AA2800002B01DD05F1310908F1010588F80090D6
:10AA38006BE0129BC3F13603F7E6089B09F1FF367A
:10AA4800B342B7BF089B9E1BF21A0C9BBFBF089668
:10AA58009B180C930026B9F1000FB9BFA8EB0905A4
:10AA6800002345464B46E2E6089E4546099FE7E631
:10AA7800089A10E71E9B012B18DC029BB3B9039BB5
:10AA8800C3F31303A3B9039B23F000431B0D1B055A
:10AA98002BB1079B08F101080133079301230893A1
:10AAA8000C9B002B7FF411AF012016E70023F6E77B
:10AAB800029BF4E73FF423AF079A1C331A449844E7
:10AAC8001D4413461AE70346F6E700BF000024407A
:10AAD800B9F1000F33DC1E9B022B30DDCDF810904E
:10AAE800049B63B931460522204600F038FB014635
:10AAF8000646504600F0F1FC00283FF75CAD1F9B6E
:10AB0800069D6FEA030B002307933146204600F0A9
:10AB18000FFB002F3FF44BAE079B2BB1BB4203D07A
:10AB28001946204600F004FB3946204600F000FB99
:10AB38003DE600263746E2E7BB4637463BE5099B3C
:10AB4800CDF81090002B7FF412AF069D3146504689
:10AB5800FFF756FA069B00F1300905F8019B049AA5
:10AB6800EB1A9A4200F38180069B012AACBF9B181E
:10AB7800013398460023079351460122204600F0EE
:10AB88005BFC3146824600F0A8FC002834DC02D188
:10AB980019F0010F30D1454615F8013C6A1E302BDB
:10ABA800B3D11546F8E73846FFE6012322E7029AB3
:10ABB800002A04DB28D11E9A32BB089A22BB002B3C
:10ABC8007FF732AF51460122204600F035FC31466E
:10ABD800824600F082FC002805DC7FF425AF19F0DE
:10ABE800010F3FF421AFB9F1390F7FF41BAF3923BF
:10ABF80008F1010808F8013C454615F8013C6A1EB1
:10AC0800392B3AD001333FE0002B08F1010505DD6F
:10AC1800B9F1390FEBD009F1010907E7069B049A4E
:10AC2800EB1A9342A84605F8019CA5D0514600238B
:10AC38000A22204600F093FA079B8246BB424FF057
:10AC48000A024FF000030799204604D100F087FA62
:10AC580007900746B1E600F082FA002307900A221F
:10AC68003946204600F07BFAF3E7514600230A22D2
:10AC7800204600F074FA824668E7069B934205D1A5
:10AC88003123069A0BF1010B13703EE71546B4E722
:10AC9800094BFFF7A3BA229B002B7FF47DAA074B31
:10ACA800FFF79CBA049B002B3FF74FAF1E9B022B6C
:10ACB8007FF74BAF14E700BFC1BC000856BD0008C2
:10ACC8008A892DE9F041054610070C465AD44B688D
:10ACD800002B05DC0B6C002B02DC0020BDE8F081AA
:10ACE800E66A002EF9D0002312F480522F682B60F8
:10ACF80033D0606DA3895A0705D56368C01A636BA2
:10AD08000BB1236CC01A00230246E66A216A284662
:10AD1800B047431CA38906D129681D294BD82B4A63
:10AD2800CA40D60747D5002262602269D90422604A
:10AD380004D5421C01D12B6803B96065616B2F6093
:10AD48000029CAD004F14403994202D0284600F0F1
:10AD58009BFC00206063BDE8F081216A012328463E
:10AD6800B047411CC6D12B68002BC3D01D2B01D086
:10AD7800162B01D12F60B0E7A38943F04003A381CC
:10AD8800BDE8F0810F69002FA7D0930718BF0023F3
:10AD98000E6808BF4B69A6EB07080F608B60B8F117
:10ADA800000F9ADD43463A46216A2846A66AB0470C
:10ADB800002807DCA38943F04003A3814FF0FF304C
:10ADC800BDE8F0810744A8EB0008E8E7010040204F
:10ADD80038B50B6905460C46DBB118B183690BB968
:10ADE80000F060F80C4B9C4209D16C68B4F90C3047
:10ADF8007BB121462846BDE83840FFF761BF074BC5
:10AE08009C4201D1AC68F1E7054B9C4208BFEC6855
:10AE1800ECE7002038BD00BF84BD0008A4BD0008D1
:10AE280064BD0008014900F0A9B800BFD9AD000809
:10AE3800002310B504460360436083608181436644
:10AE4800C281036143618361194608225C30FEF7C1
:10AE58007CFA054B24626362044BA362044BE362F1
:10AE6800044B236310BD00BF81BA0008A3BA0008D1
:10AE7800DBBA0008FFBA000870B568254A1E5543BA
:10AE88000E4605F1740100F04BFC044640B1002168
:10AE980080E842000C30A06005F16802FEF755FA20
:10AEA800204670BD836910B5044633BB8364C36410
:10AEB8000365124B124A1B688262984204BF012341
:10AEC800836100F01FF86060204600F01BF8A06066
:10AED800204600F017F80022E06004216068FFF7C0
:10AEE800A7FF01220921A068FFF7A2FF0222122171
:10AEF800E068FFF79DFF0123A36110BD20BD000896
:10AF08002DAE0008F8B51C4B07461E68B36913B987
:10AF18003046FFF7C7FF4836B4687368013B03D56E
:10AF2800336833B13668F7E7B4F90C506DB168345B
:10AF3800F4E704213846FFF79FFF30600028F1D17D
:10AF48000C2304463B602046F8BD4FF6FF73E381AF
:10AF580001236566A3812560A5606560256165613B
:10AF6800A5610822294604F15C00FEF7EEF9656345
:10AF7800A563A564E564E6E720BD00082DE9F8436C
:10AF880080468946002600F1480414B93046BDE8D9
:10AF9800F883A5686768013F01D52468F5E7AB89A0
:10AFA800012B07D9B5F90E30013303D029464046A5
:10AFB800C84706436835EEE7044B1B68186A044B1C
:10AFC800002808BF1846F030704700BF4C02002028
:10AFD800B002002070B50E46B1F90E1090B00029ED
:10AFE80014461D4607DA00232B60B3891A0610D4CD
:10AFF8004FF480630EE001AA00F0A4FD0028F2DB04
:10B00800029A02F47042A2F500535A425A412A6049
:10B01800EEE740230020236010B070BD8B8973B524
:10B028009D0706460C4607D504F1470323602361B4
:10B038000123636102B070BD01AB6A46FFF7CAFF26
:10B0480000990546304600F06BFB48B9B4F90C305E
:10B058009A05EFD423F0030343F00203A381E3E747
:10B068000D4BB362A389206043F08003A381009B4A
:10B0780020616361019B5BB1B4F90E10304600F0AA
:10B0880073FD28B1A38923F0030343F00103A381CF
:10B09800A3891D43A581CDE72DAE0008024B0146CB
:10B0A800186800F03DBB00BF4C02002010B5C9B2C3
:10B0B80002449042034601D1002010BD1C780130A3
:10B0C8008C42F6D1184610BD70B5456A04460E4646
:10B0D8003DB91020FFF7E2FF6062456085600560BA
:10B0E800C560656AEB6883B1636ADB6853F826005C
:10B0F800B8B9012101FA06F56A1D9200204600F050
:10B10800B4FA60B1466085600EE021220421204631
:10B1180000F0ABFA636AE860DB68002BE4D100203A
:10B1280070BD026843F8262000230361C36070BD28
:10B1380070B5446A06460D463CB91020FFF7AEFFCD
:10B148007062446084600460C4603DB1736A6A6878
:10B15800DB6853F82210296043F8225070BD2DE9AE
:10B16800F0411F4606460C4600230D6901F1140EF6
:10B17800DEF80000013381B202FB0171000C0F0CF4
:10B1880002FB007089B201EB00419D424FEA104773
:10B198004EF8041BECDCD7B1A3689D4212DB616852
:10B1A80030460131FFF790FF8046226904F10C0117
:10B1B800023292000C30FEF7BDF821463046FFF708
:10B1C800B7FF444604EB850301355F6125612046DE
:10B1D800BDE8F081020C12040346B2B90304102042
:10B1E80013F07F4F04BF1B02083013F0704F04BFE9
:10B1F8001B01043013F0404F04BF9B000230002BAA
:10B2080006DB5B0003D5013070470020E8E720200B
:10B2180070470368014613F007020BD0DA0723D4FE
:10B22800980749BF5B089B0801200B605CBF0B6057
:10B238000220704798B2A8B910201B0C13F0FF0F1A
:10B2480004BF1B0A08301A0704BF1B0904309A07F9
:10B2580004BF9B080230DA0702D45B0806D001302D
:10B268000B6070471046E9E70020704720207047C0
:10B2780010B50C460121FFF727FF01224461026146
:10B2880010BD2DE9F74F14460A69236989469A4289
:10B29800BEBF0B46A1461C46D9F81070D4F810A0C2
:10B2A800D9F80830D9F8041007EB0A069E42C8BF3F
:10B2B8000131FFF709FF00F114052B46002205EBC9
:10B2C8008608434516D304F1140209F1140102EB70
:10B2D8008A0301EB87070193019C134694420CD81B
:10B2E800002E03DD58F8043D002B54D0066103B04E
:10B2F800BDE8F08F43F8042BE3E7B3F800A004326D
:10B30800BAF1000F20D0AE4689464FF0000C59F82C
:10B31800044BBEF800B0A3B20AFB03B34FEA144BC8
:10B32800DEF8004063444FEA144C0AFB0BC404EBFC
:10B3380013449BB243EA04434F454FEA144C4EF87A
:10B34800043BE4D8CEF800C032F8029CB9F1000FF3
:10B358001FD0AE468C464FF0000A2B68BCF8004060
:10B36800BEF802B09BB209FB04B4A24443EA0A4304
:10B378004EF8043B5CF8043BBEF800401B0C09FB8C
:10B388000343674503EB1A434FEA134AE6D8CEF85E
:10B3980000300435A0E7013EA2E700002DE9F8439C
:10B3A800154612F0030206460F4607D0214C013A13
:10B3B800002354F82220FFF7D2FE0746AD1035D0FF
:10B3C800746A3CB91020FFF769FE706244608460BB
:10B3D8000460C460D6F82480D8F808404CB940F21C
:10B3E80071213046FFF744FF00230446C8F80800DF
:10B3F80003604FF00008EB070AD53946224630466D
:10B40800FFF73FFF814639463046FFF791FE4F462A
:10B418006D100BD0206838B9224621463046FFF718
:10B4280030FF2060C0F800800446E4E73846BDE8F5
:10B43800F88300BFB8BE00082DE9F0470C46074660
:10B44800164623694FEA621A0AEB03094968A3689A
:10B4580009F10105AB4231DB3846FFF735FE002222
:10B468008046114600F1140352452ADB20692AEA76
:10B47800EA7A04F1140116F01F0203EB8A0301EBC8
:10B48800800E22D00020C2F1200C0E689640304376
:10B4980043F8040B51F8040B8E4520FA0CF0F4D84D
:10B4A800186008B109F10205013D3846C8F8105086
:10B4B8002146FFF73DFE4046BDE8F08701315B00BD
:10B4C800C8E743F822100132CEE7043B51F8042BB9
:10B4D8008E4543F8042FF9D8E6E703690A6930B5C1
:10B4E8009B1A0CD19200143014318418114454F86A
:10B4F800045D51F8042D954203D005D30123184665
:10B5080030BDA042F3D3FAE74FF0FF33F7E72DE958
:10B51800F0470D460746114628461446FFF7DDFF5B
:10B52800061E08D131463846FFF7CEFD0123466195
:10B538000361BDE8F087A4BF23462C4638466168FE
:10B54800A6BF1D4600260126FFF7BEFD4FF0000CE2
:10B55800C6602B69266904F1140205F1140902EB8F
:10B56800860709EB830800F1140152F804AB59F877
:10B57800045B1FFA8AF36344ACB21B1B2C0CC4EBAC
:10B588001A4404EB23449BB24FEA244CC84543EACF
:10B598000444964641F8044BE7D8BE4505D351F814
:10B5A800043D8BB10661BDE8F0875EF8044BA2B29A
:10B5B8006244131403EB144392B242EA03424FEA83
:10B5C800234C41F8042BE8E7013EE8E72DE9F34175
:10B5D8001C4601219046089E099DFFF775FDC4F39E
:10B5E8001302C4F30A54074634BB0192B8F1000FA2
:10B5F80027D002A840F8088DFFF70BFE0099F0B19C
:10B60800019AC0F1200302FA03F30B43C2407B61A5
:10B618000192019B002B14BF02210121BB613961FA
:10B62800C4B1A4F2334404443460C0F13500286046
:10B63800384602B0BDE8F08142F48012D5E779615E
:10B64800E7E701A8FFF7E5FD0121019B39617B616F
:10B658002030E5E7A0F2324007EB8103306018693B
:10B66800FFF7B8FDC0EB4110E1E738B502FB01F484
:10B67800214600F055F8054618B122460021FDF78D
:10B6880064FE284638BD000038B50546002943D079
:10B6980051F8043C0C1F002BB8BFE41800F098FACE
:10B6A8001E4A1368104633B9636014602846BDE823
:10B6B800384000F08EBAA3420BD921686218934231
:10B6C80001BF1A685B685218226063600460EDE786
:10B6D80013465A680AB1A242FAD919685818A04202
:10B6E8000BD120680144581882421960DED11068D5
:10B6F8005268014419605A60D8E702D90C232B60BC
:10B70800D4E7206821188A4201BF116852680918D5
:10B71800216062605C60C9E738BD00BF700400202A
:10B7280070B5CD1C25F0030508350C2D38BF0C2548
:10B73800002D064601DBA94203D90C233360002003
:10B7480070BD00F045FA234A1468214691B9224C8D
:10B7580023681BB9304600F07FF92060294630463F
:10B7680000F07AF9431C26D10C233046336000F0F0
:10B7780030FAE4E70B685B1B1AD40B2B0FD90B606C
:10B78800CC18CD50304600F024FA04F10B00231DEC
:10B7980020F00700C31A1BD05A42E25070BD8C42F9
:10B7A8000BBF63684B681360636018BF0C46E9E71A
:10B7B8000C464968CAE7C41C24F00304A04205D01B
:10B7C800211A304600F048F90130CDD02560D9E77C
:10B7D80070BD00BF7004002074040020936810B48A
:10B7E800013B002B936008DA9469A34202DBCBB2D9
:10B7F8000A2B02D110BCFEF743BB1368581C10601B
:10B808001970C8B210BC7047F8B506460F46144602
:10B81800D518AC4201D1002007E03A4614F8011BC4
:10B828003046FFF7DBFF431CF3D1F8BD2DE9F04F9D
:10B838009DB00C4617460393064618B183690BB9A9
:10B84800FFF730FB7C4B9C4257D17468A3891807DB
:10B858005DD52369002B5AD00023099320238DF846
:10B86800293030234FF0010B8DF82A30B846454671
:10B8780015F8013B002B55D1B8EB070A0BD05346FE
:10B888003A4621463046FFF7BFFF013000F0C4803A
:10B89800099B5344099398F80030002B00F0BC80B2
:10B8A80000234FF0FF3204930793059206938DF817
:10B8B80053301A93052229786048FFF7F7FB05F102
:10B8C8000108049B002831D1D90644BF20228DF8F5
:10B8D80053201A0744BF2B228DF853202A782A2A8E
:10B8E8002CD000210A20079AA84698F80030013584
:10B8F800303B092B6DD971B326E0514B9C4201D1E5
:10B90800B468A3E74F4B9C4208BFF4689EE7214602
:10B918003046FEF707FB00289ED04FF0FF301DB0E1
:10B92800BDE8F08F252BA7D0A846A0E7434A454697
:10B93800801A0BFA00F018430490BBE7039A111D14
:10B9480012680391002A01DB079204E0524243F097
:10B9580002030792049398F800302E2B10D198F820
:10B96800013008F101012A2B37D1039B08F10208A5
:10B978001A1D1B680392002BB8BF4FF0FF330593C5
:10B98800314D032298F800102846FFF78FFB40B18D
:10B998004023401B03FA00F0049B08F1010803430D
:10B9A800049398F800100622284808F101078DF83A
:10B9B8002810FFF77BFB002834D0254B03BB039BE3
:10B9C800073323F0070308330393099B4B44099378
:10B9D8004CE700FB0232012186E700230A251846BE
:10B9E8000593884698F800200131303A092A03D98E
:10B9F800002BC5D00590C3E705FB00200123F0E725
:10BA080003AB00932246134B04A93046FDF736FDDD
:10BA1800B0F1FF3F8146D8D1A3895B063FF57DAFE2
:10BA280009987CE703AB009322460A4B04A93046E9
:10BA3800FDF7D4FFECE700BF84BD0008C4BE0008D2
:10BA4800A4BD000864BD0008CABE0008CEBE000838
:10BA58008594000811B8000838B50023054C054640
:10BA680008462360FCF7DCFD431C02D1236803B1C0
:10BA78002B6038BDE017002010B50C46B1F90E1048
:10BA880000F0A8F80028ABBF636DA3891B1823F446
:10BA98008053ACBF6365A38110BD2DE9F0411F46FB
:10BAA8008B890546DB050C46164605D50223002280
:10BAB800B1F90E1000F068F8A389324623F48053D8
:10BAC800A381B4F90E103B462846BDE8F04100F0CA
:10BAD80017B810B50C46B1F90E1000F055F8431C14
:10BAE800A38915BF606523F4805343F48053A38171
:10BAF80018BFA38110BDB1F90E1000F013B80000F3
:10BB080038B50546084611460022054C22601A46FB
:10BB1800FCF7CEF8431C02D1236803B12B6038BD73
:10BB2800E017002038B50023054C05460846236079
:10BB3800FCF790FD431C02D1236803B12B6038BD8C
:10BB4800E017002038B50023064C05460846114684
:10BB58002360FCF782FD431C02D1236803B12B60EC
:10BB680038BD00BFE017002038B50023054C054656
:10BB780008462360FCF776FD431C02D1236803B115
:10BB88002B6038BDE017002038B505460846114639
:10BB98000022054C22601A46FCF766FD431C02D1C0
:10BBA800236803B12B6038BDE017002082B001B9CB
:10BBB80001A942B14BB113780B601278101C18BF61
:10BBC800012002B070471046FBE76FF00100F8E76C
:10BBD8007047704738B50546084611460022054C9F
:10BBE80022601A46FCF70EFD431C02D1236803B1FC
:10BBF8002B6038BDE017002049B1FF2A8BBF8A238C
:10BC08000A700360012088BF4FF0FF307047084674
:10BC180070470000F8B500BFF8BC08BC9E467047E6
:0CBC2800F8B500BFF8BC08BC9E46704791
:10BC380002030405060708090A0B0C0D0E0F101065
:10BC480002030405060708090A0B0C0D0E0F101055
:10BC5800457261736572204572726F720D0057727A
:10BC6800697465204572726F722025640D0A002A76
:10BC78002A2A2A2A2A2A2A2A2A2A2A2A2A2A2A2A1C
:10BC88002A2A2A2A2A2A2A2A2A2A2A2A2A2A2A2A0C
:10BC98002A2A2A2A2A2A2A0D004D414F2050726F3B
:10BCA8006A6563740D0031373A32373A3439004ADD
:10BCB800756E2020352032303230004275696C6450
:10BCC8002061742025732025730D0A00436F707955
:10BCD80072696768742028632920323032302E2038
:10BCE800424C554543454C4C0D00000000000000F7
:10BCF8000000010203040607080900000000010211
:10BD0800030425303278200052657365742053741B
:10BD1800617274200D00000050020020494E460058
:10BD2800696E66004E414E006E616E0030313233EE
:10BD3800343536373839414243444546003031328C
:10BD48003334353637383961626364656600496E65
:10BD580066696E697479004E614E0000000000004B
:10BD680000000000000000000000000000000000CB
:10BD780000000000000000000000000000000000BB
:10BD880000000000000000000000000000000000AB
:10BD9800000000000000000000000000000000009B
:10BDA800000000000000000000000000000000008B
:10BDB800000000000000000000000000000000007B
:10BDC8000080E03779C34143176E05B5B5B893468F
:10BDD800F5F93FE9034F384D321D30F94877825A5B
:10BDE8003CBF737FDD4F1575000000000000F03F79
:10BDF800000000000000244000000000000059403E
:10BE08000000000000408F40000000000088C34090
:10BE180000000000006AF8400000000080842E4105
:10BE280000000000D01263410000000084D7974151
:10BE38000000000065CDCD41000000205FA0024257
:10BE4800000000E876483742000000A2941A6D42CC
:10BE5800000040E59C30A2420000901EC4BCD642BF
:10BE680000003426F56B0C430080E03779C341436A
:10BE780000A0D8855734764300C84E676DC1AB43E0
:10BE8800003D9160E458E143408CB5781DAF1544FE
:10BE980050EFE2D6E41A4B4492D54D06CFF08044D9
:10BEA800F64AE1C7022DB544B49DD9794378EA44EE
:10BEB80005000000190000007D000000232D302B34
:10BEC8002000686C4C006566674546470043005093
:10BED8004F534958002E00002020202020202020E9
:10BEE8002028282828282020202020202020202022
:10BEF8002020202020202020881010101010101042
:10BF08001010101010101010040404040404040489
:10BF1800040410101010101010414141414141011A
:10BF280001010101010101010101010101010101F9
:10BF38000101011010101010104242424242420208
:10BF480002020202020202020202020202020202C9
:10BF58000202021010101020000000000000000073
:10BF680000000000000000000000000000000000C9
:10BF780000000000000000000000000000000000B9
:10BF880000000000000000000000000000000000A9
:10BF98000000000000000000000000000000000099
:10BFA8000000000000000000000000000000000089
:10BFB8000000000000000000000000000000000079
:10BFC8000000000000000000000000000000000069
:08BFD800000000000000000061
:04BFE0000D42000806
:04BFE400E941000827
:10BFE80001000000100000000014014000080000DB
:10BFF8000014014000040000001801400400000083
:10C008000014014000080000001401400004000072
:10C01800001801400800000000140140000800005A
:10C028000014014000040000001801401000000046
:10C038000014014000080000001401400004000042
:10C048000018014020000000001401400008000012
:10C0580000140140000400000018014040000000E6
:10C068000014014000080000001401400004000012
:10C0780000100140002000000014014000080000EA
:10C088000014014000040000001C014010000000E2
:10C0980000140140000800000014014000040000E2
:10C0A800001C0140200000000014014000080000AE
:10C0B8000014014000040000001C01404000000082
:10C0C80000140140000800000014014000040000B2
:10C0D800001C01408000000000140140000800001E
:10C0E8000014014000040000001C01400001000091
:10C0F8000014014000080000001401400004000082
:10C10800001C014000020000001401400100000072
:10C11800001401401000000000140140020000005B
:10C12800001401400100000000140140400000001C
:10C13800001401400200000000140140010000004A
:10C148000014014008000000001401400200000033
:10C158000014014001000000002001400020000000
:10C16800001401400200000000140140010000001A
:10C178000014014004000000001401400200000007
:10C1880000140140010000000014014020000000DC
:10C1980000140140020000000008014000010000F6
:10C1A8000008014000010000001C014001000000DF
:10C1B80000080140000100000008014000010000E3
:10C1C800001C0140020000000008014000010000BE
:10C1D8000008014000010000000C014008000000B8
:10C1E80000080140000100000008014000010000B3
:10C1F800000C01401000000000A24A040014014095
:10C20800000200000014014000010000001001407D
:10C2180080000000001401400002000000140140EA
:10C228000001000000100140400000005002002002
:10C238000000000084BD0008A4BD000864BD00081B
:10C2480000000000000000000000000000000000E6
:10C2580000000000000000000000000000000000D6
:10C2680000000000000000000000000000000000C6
:10C2780000000000000000000000000000000000B6
:10C2880000000000000000000000000000000000A6
:10C298004300000000000000000000000000000053
:10C2A8000000000000000000000000000000000086
:10C2B8004300000000000000000000000000000033
:10C2C8000000000000000000000000000000000066
:10C2D8004300000000000000000000000000000013
:10C2E8000000000000000000000000000000000046
:10C2F80043000000000000000000000000000000F3
:10C308000000000000000000000000000000000025
:10C3180043000000000000000000000000000000D2
:10C328000000000000000000000000000000000005
:10C3380043000000000000000000000000000000B2
:10C3480000000000000000000000000000000000E5
:10C358004300000000000000000000000000000092
:10C3680000000000000000000000000000000000C5
:10C3780001BC0008B5BB000800000000DFBE0008D3
:10C38800DDBE000876BC000876BC000876BC000854
:10C3980076BC000876BC000876BC000876BC0008AD
:10C3A80076BC000876BC0008FFFFFFFFFFFFFFFF19
:10C3B800FFFFFFFFFFFF0000010041534349490011
:10C3C8000000000000000000000000000000000065
:10C3D80000000000000000000000415343494900EC
:10C3E8000000000000000000000000000000000045
:0CC3F80000000000000000000000000039
:040000050800929DC0
:00000001FF
